:020000040800F2
:1000000000100020A9410008F5410008F541000852
:1000100000000000000000000000000000000000E0
:10002000000000000000000000000000F541000892
:100030000000000000000000F54100083D3F0008FE
:10004000F5410008F5410008F5410008F5410008B8
:10005000F5410008193F0008F5410008F541000886
:10006000F5410008F5410008F5410008F541000898
:10007000F5410008F5410008F5410008F541000888
:10008000F5410008F541000800000000F5410008B6
:10009000F5410008F5410008F5410008B1400008AD
:1000A000F5410008F5410008F5410008F541000858
:1000B000F541000800000000F541000800000000C4
:1000C0005FF808F180B582B000AF021CFB1D1A700A
:1000D000FB1D1B78002B06D0074B074A1268012135
:1000E0000A431A6005E0044B034A126801218A435F
:1000F0001A60BD4602B080BD0010024080B582B0DB
:1001000000AF78600A1CFB1C1A70FB1C1B78002BCC
:1001100006D0084B074A51697A680A435A6106E0DB
:10012000044B044A52697968C9430A405A61BD4682
:1001300002B080BD0010024080B582B000AF786090
:100140000A1CFB1C1A70FB1C1B78002B06D0084BEA
:10015000074A91697A680A439A6106E0044B044AA7
:1001600092697968C9430A409A61BD4602B080BD70
:100170000010024080B582B000AF78600A1CFB1C02
:100180001A70FB1C1B78002B06D0084B074AD1685D
:100190007A680A43DA6006E0044B044AD268796858
:1001A000C9430A40DA60BD4602B080BD001002407B
:1001B00080B582B000AF78600A1CFB1C1A70FB1C73
:1001C0001B78002B06D0084B074A11697A680A434E
:1001D0001A6106E0044B044A12697968C9430A406F
:1001E0001A61BD4602B080BD0010024080B582B0E9
:1001F00000AF786039607A683B68101C191C04F005
:10020000DBFB044B1B681A1D024B1A60BD4602B093
:1002100080BDC0466800002080B582B000AF786025
:10022000024B00221A60BD4602B080BD680000206B
:1002300080B588B000AF80239B02181C0121FFF716
:100240005DFF80235B01181C0121FFF775FF3B1D3B
:1002500020221A603B1D02221A713B1D03225A7193
:100260003B1D00229A713B1D0122DA719023DA05B1
:100270003B1D101C191C04F083FE3B1D40221A601C
:100280009023DA053B1D101C191C04F079FE3B1D60
:1002900080221A609023DA053B1D101C191C04F003
:1002A0006FFE3B1D414A1A603B1D01221A713B1D26
:1002B00000229A713B1D0122DA713B1D01225A7105
:1002C0009023DA053B1D101C191C04F059FE9023E5
:1002D000DB05181C0521002204F03CFF9023DB0500
:1002E000181C0621002204F035FF9023DB05181CA2
:1002F0000721002204F02EFF2D4B181C04F074FC83
:100300000C23FB1800221A800C23FB1882225200B7
:100310005A800C23FB18E022D2009A800C23FB1891
:100320000022DA800C23FB1800221A810C23FB1810
:10033000802292005A810C23FB1800229A810C2300
:10034000FB180022DA810C23FB1807221A82184AB4
:100350000C23FB18101C191C04F072FC144A802397
:100360005B01101C191C04F00DFD9023DB05181C0B
:100370000121012204F0D2FE9023DA0580235B00E4
:10038000101C191C012204F0C9FE9023DA058023F9
:100390001B02101C191C012204F0C0FE044B181C87
:1003A000012104F0CFFCBD4608B080BD01810000F2
:1003B0000030014080B582B000AF786000F0E6F90F
:1003C000002000F0A9F9D82000F0B8F97A68FF23DE
:1003D0001B0413401B0CDBB2181C00F0AFF97A6849
:1003E000FF231B0213401B0ADBB2181C00F0A6F906
:1003F0007B68DBB2181C00F0A1F9012000F08CF939
:1004000000F0D2F9BD4602B080BDC04680B584B0D0
:1004100000AFF860B960BB1D1A8000F0B7F900208A
:1004200000F07AF9022000F089F9BA68FF231B0472
:1004300013401B0CDBB2181C00F080F9BA68FF23D4
:100440001B0213401B0ADBB2181C00F077F9BB68D3
:10045000DBB2181C00F072F907E0FB681B78181C6F
:1004600000F06CF9FB680133FB60BB1D1B88BA1DF3
:10047000591E1180002BF0D1012000F04DF900F041
:1004800093F9BD4604B080BD80B586B000AFF8607A
:10049000B960BB1D1A801723FB1800221A7016239F
:1004A000FB1800221A701523FB1800221A7014235F
:1004B000FB1800221A701323FB1800221A70152350
:1004C000FB18BA681A701423FB181522BA18127890
:1004D00052421A70BB1D1B881B0A9AB21723FB18C5
:1004E0001A701623FB18BA1D12881A701523FB18F0
:1004F0001B78002B35D11723FB181B78002B09D153
:10050000F968BA68BB1D1B88081C111C1A1CFFF770
:100510007DFFC1E010E0F968BA6880235B00081C29
:10052000111C1A1CFFF772FFBB680133FF33BB605D
:10053000FB680133FF33FB601723FB181B7817227E
:10054000BA18591E1170002BE5D11623FB181B7821
:100550009BB2F968BA68081C111C1A1CFFF756FFF9
:100560009AE01723FB181B78002B3ED11623FA18AC
:100570001423FB1812781B789A422CD91323FB18EA
:100580001622B9181422BA18097812788A1A1A7021
:100590001423FB181B789BB2F968BA68081C111C5D
:1005A0001A1CFFF733FF1423FB181B78BA68D31803
:1005B000BB601423FB181B78FA68D318FB60132365
:1005C000FB181B789BB2F968BA68081C111C1A1C2E
:1005D000FFF71CFF60E0F968BA68BB1D1B88081CA8
:1005E000111C1A1CFFF712FF56E01423FB181B788E
:1005F0009AB2BB1DB91D09888A1A1A80BB1D1B88B7
:100600001B0A9AB21723FB181A701623FB18BA1D7F
:1006100012881A701423FB181B789BB2F968BA6809
:10062000081C111C1A1CFFF7F1FE1423FB181B7881
:10063000BA68D318BB601423FB181B78FA68D31868
:10064000FB6010E0F968BA6880235B00081C111C8D
:100650001A1CFFF7DBFEBB680133FF33BB60FB688E
:100660000133FF33FB601723FB181B781722BA18DE
:10067000591E1170002BE5D11623FB181B78002B97
:100680000AD01623FB181B789BB2F968BA68081CBD
:10069000111C1A1CFFF7BAFEBD4606B080BDC0464D
:1006A00080B584B000AFF860B960BB1D1A8000202F
:1006B00000F032F8032000F041F8BA68FF231B0471
:1006C00013401B0CDBB2181C00F038F8BA68FF238B
:1006D0001B0213401B0ADBB2181C00F02FF8BB688A
:1006E000DBB2181C00F02AF809E0A52000F026F87B
:1006F000031C1A1CFB681A70FB680133FB60BB1DEE
:100700001B88BA1D591E1180002BEED1012000F06C
:1007100003F8BD4604B080BD80B582B000AF021CB6
:10072000FB1D1A709023DA05FB1D1B78101C01219C
:100730001A1C04F0F3FCBD4602B080BD80B582B047
:1007400000AF021CFB1D1A70C0460F4B181C022183
:1007500004F05EFB031EF8D00B4AFB1D1B78101C37
:10076000191C04F02DFBC046074B181C012104F096
:100770004FFB031EF8D0044B181C04F037FB031C7E
:10078000181CBD4602B080BD0030014080B500AFEE
:100790000020FFF7C1FF0620FFF7D0FF0120FFF781
:1007A000BBFFBD4680BDC04690B583B000AFFB1D0A
:1007B00000221A700020FFF7AFFF0520FFF7BEFFF1
:1007C000FC1DA520FFF7BAFF031C2370FB1D1B783F
:1007D00001221340F4D10120FFF79EFFBD4603B074
:1007E00090BDC046B0B582B000AF021C3960FB1DA1
:1007F0001A70FB1D1B787F2B2FD92D4CFB1D1B78EE
:100800001A1C0F231340083B9908294AFB1D1B782B
:10081000181C0F230340083B9B0806339B00D3188A
:100820005B68FA1D1278101C03220240D200101CD3
:10083000FF228240D2431A403B689B01FF200340C5
:10084000F81D0078051C03202840C00083401A438F
:100850008B1D9B00E3185A6026E0164CFB1D1B788D
:100860005BB29B081349FA1D127852B29208C0324B
:1008700092005258F91D0978081C03210140C90053
:10088000081CFF218140C94311403A689201FF20B2
:100890000240F81D0078051C03202840C00082405B
:1008A0000A43C0339B001A51BD4602B0B0BDC046DA
:1008B00000ED00E000E100E080B582B000AF7860BC
:1008C0007B680E4A934201D9012312E00C4B7A68EF
:1008D0001202120A013A5A6001235B42181C0321DA
:1008E000FFF780FF064B00229A60054B07221A6033
:1008F0000023181CBD4602B080BDC046FFFFFF00AC
:1009000010E000E080B586B000AF8023DB02181C49
:100910000121FFF7F3FB1023FB1802221A601023BA
:10092000FB1800221A711023FB1803225A7110239E
:10093000FB180122DA711C4A1023FB18101C191C29
:1009400004F01EFB01200121FFF7F6FB012001212D
:1009500004F0EAFF0823FB1802221A600823FB18A0
:1009600000221A710823FB180C225A710823FB1865
:1009700001229A710823FB18181C04F039FF3B1D53
:1009800005221A703B1D00225A703B1D01229A70ED
:100990003B1D181C05F010F80120012104F0C4FFD4
:1009A000BD4606B080BDC0460004004880B500AF1B
:1009B0000120FFF787FB042005F052F8FA235B01C2
:1009C000181CFFF779FFBD4680BDC04680B500AF5B
:1009D0004E4B1B684E4A181C111CFFF707FC4B4B73
:1009E0001B684C4A181C111CFFF700FC474B1B6886
:1009F000494A181C111CFFF7F9FB444B1B68474A76
:100A0000181C111CFFF7F2FB404B1B68444A181CD2
:100A1000111CFFF7EBFB3D4B1B68424A181C111CD5
:100A2000FFF7E4FB394B1B683F4A181C111CFFF70A
:100A3000DDFB364B1B683D4A181C111CFFF7D6FB2B
:100A4000324B1B683A4A181C111CFFF7CFFB2F4B87
:100A50001B68384A181C111CFFF7C8FB2B4B1B687E
:100A6000354A181C111CFFF7C1FB284B1B68334A81
:100A7000181C111CFFF7BAFB244B1B68304A181CCA
:100A8000111CFFF7B3FB214B1B682E4A181C111CCD
:100A9000FFF7ACFB1D4B1B682B4A181C111CFFF702
:100AA000A5FB1A4B1B68294A181C111CFFF79EFB5B
:100AB000164B1B68264A181C111CFFF797FB134B9B
:100AC0001B68244A181C111CFFF790FB0F4B1B6876
:100AD000214A181C111CFFF789FB0C4B1B681F4A8D
:100AE000181C111CFFF782FB084B1B681C4A181CC2
:100AF000111CFFF77BFB054B1A6884239B05101C18
:100B0000191CFFF773FBBD4680BDC046FC020020E8
:100B10000300001FD87F607F80204041D87F2043A2
:100B200080200045D87F804780206049D87F004AD8
:100B30008020E04BD87F804C8020604ED87F404B97
:100B40008020204D0000EC7F407C40558007EC7FEA
:100B5000C0034055000FEC7F400B40558016EC7FE2
:100B6000C0124055F0B587B004AFC54B1B78012BC0
:100B70002FD1C44B1F221A60C34B32221A60C34BC1
:100B800032221A60C24B0F221A60C24B7C221A70AA
:100B9000C14B00221A70C14B00221A70C04B0122B7
:100BA0001A70C04B00221A60BF4B1B78DBB2032BBC
:100BB00004D0BD4B1B78DBB2062B07D1BB4B1B68A7
:100BC000BB4A181C111C012203F08EFDAC4B002205
:100BD0001A70B64B1B68B74A181C111C03F028FD8D
:100BE000031C1A1CAC4B1A70B04B1B68B24A181C81
:100BF000111C03F05DFD031CDB0FDAB2A84B1A7069
:100C0000A54B1A78A34B1A70A34B1B78F92B02D172
:100C1000A14B00221A70A04B1B78002B02D19D4BD8
:100C20007C221A709E4B1B78012B0FD19B4B1B789B
:100C3000002B0BD09B4B1B685A1C9A4B1A60994B8C
:100C40001B68182B02DD974B00221A60974B1B681C
:100C5000181C04F0B3FD954B1A6880239B04101CEC
:100C6000191CFFF7C3FA914B1B68944A181C111CFE
:100C7000FFF7BCFA8D4B1B68914A181C111CFFF73B
:100C8000B5FA884B1B68834A11788E4AD154854B3C
:100C90001B6801338B4A0021D154844B1A68A0236E
:100CA0005B05101C191CFFF7A1FA804B1A68864BD4
:100CB0001B68002B00DA01335B10191C714B1C6898
:100CC000C023DB0000937F4B0193101C2822231CC0
:100CD00004F0D2FA754B1B687C4A181C111CFFF7F4
:100CE00085FA7B4B82221A60704B1B68794A181C6C
:100CF000111C04F087FB6D4B1A68FF231B02101CAC
:100D0000191C04F07DFC694B1E68614B1D68704B1B
:100D10001C685D4B1A68131C9B009B185B007B6072
:100D20005A4B1968574B1A685B4B1B789BB2C02013
:100D3000C00003439BB2009101920293664B039360
:100D4000301C291C221C7B6804F0E4FC574B1B68F8
:100D5000624A181C111C04F053FC4C4B1A684C4B93
:100D60001B68D2185A4B1B68D218594B1A604F4B4C
:100D70001E68474B1D68564B1C68434B1A68131C72
:100D80009B009B185B007B60404B19683D4B1A68C9
:100D9000414B1B789BB2C020C00003439BB2009123
:100DA000019202934E4B0393301C291C221C7B683A
:100DB00004F0B0FC3D4B1B684A4A181C111C04F09F
:100DC0001FFC324B1A68324B1B68D218404B1B6811
:100DD000D2183F4B1A60354B1E682D4B1D683C4B9B
:100DE0001C68294B1A68131C9B009B185B007B60D6
:100DF000264B1968234B1A68274B1B789BB2C020DF
:100E0000C00003439BB2009101920293364B0393BF
:100E1000301C291C221C7B6804F07CFC1B4B1A68CC
:100E20001B4B1B68D2182A4B1B68D218284B1A6020
:100E30001E4B1B682D4A181C111CFFF7D7F9164BC7
:100E40001B78202B56D1194B1868114B1968204B71
:100E50001C680D4B1A68131C9B009B185B001D1C23
:100E60000A4B1A68074B1B6800920193E023DB00D2
:100E700002931F4B0393221C2B1C04F0E3FA55E052
:100E8000F802002070000020B00000207400002054
:100E900038030020E00200209C0000209D0000207C
:100EA000B40000208000002085000020FC0200200B
:100EB000082130002C2130008C2130000700002652
:100EC000FFFFFF04B8000020000000200100001414
:100ED00000030020804040003C5F0008FFFF00004E
:100EE000485F000800FFFF00545F00082000000377
:100EF0005C5F0008B74B1868B74B1968B74B1C68A4
:100F0000B74B1A68131C9B009B185B001D1CB54B4C
:100F10001A68B54B1B6800920193C023DB00029353
:100F2000B24B0393221C2B1C04F08CFAAB4B822295
:100F30001A60A84B1868AA4B1A68131C9B009B18D0
:100F40005B009E18A54B1D68A54B1A68131C5B001F
:100F50009C18A44B1968A44B1A68A54B1B789BB22C
:100F6000009101920293A34B0393311C2A1C231C72
:100F700004F0D0FB9B4B1A68974B1B68D218974B19
:100F80001B68D218954B1A60924B1868944B1A68DC
:100F9000131C9B009B185B009E18904B1D68904B88
:100FA0001A68131C5B009C188E4B19688E4B1A68CC
:100FB0008F4B1B789BB20091019202938E4B03934F
:100FC000311C2A1C231C04F0A5FB864B1A68824B9B
:100FD0001B68D218814B1B68D218804B1A607D4B5E
:100FE00018687F4B1A68131C9B009B185B009E18A7
:100FF0007A4B1D687A4B1A68131C5B009C18794B5E
:101000001968794B1A687A4B1B789BB20091019250
:1010100002937A4B0393311C2A1C231C04F07AFBA5
:10102000704B1A686C4B1B68D2186C4B1B68D2183B
:101030006A4B1A60674B1B68714A181C111CFFF73A
:10104000D5F8644B1868664B1A68131C9B009B18F4
:101050005B009E18614B1D68614B1A68131C5B0096
:101060009C18604B1968604B1A68614B1B789BB2E7
:10107000009101920293634B0393311C2A1C231CA1
:1010800004F048FB534B1B685F4A181C111CFFF708
:10109000ADF85E4B00221A705C4B181C04F0BAFECF
:1010A000031C1A1C594BD218594B111C1A1C0E2325
:1010B000081C111C1A1C04F06FFE564B1B68181CF0
:1010C000642104F0E7FC031C01331A1C4F4B181C6D
:1010D000111C03F0C5FC4D4B181C04F09BFE031CB7
:1010E0001A1C4A4BD2184C4B111C1A1C0223081C08
:1010F000111C1A1C04F050FE364B1868474B196837
:10110000474B1B680C3B1A1C80231B0100933F4B71
:101110000193142304F0B0F8424B1B78DBB2022B8E
:101120000ED0404B1B78DBB2032B09D03D4B1B7814
:10113000DBB2052B04D03B4B1B78DBB2062B2DD149
:10114000244B1B68384A181C111CFFF74FF8214B21
:101150001B68364A181C111CFFF748F81D4B18680D
:101160002E4B1B68413B191C2D4B1B682A3B1A1C3C
:101170001E23009314230193002302932C4B03930B
:101180003C2304F05FF9134B1B682A4A181C111CFE
:1011900003F04EFA031C1A1C274B1A700D4B1B68E8
:1011A000181C0021FFF722F80A4B1B68181C04F0DA
:1011B000F9F8084B1B68181CFFF72EF8054B1B6845
:1011C000181C03F0D1FB0A4B1A781C4B1A70BD4651
:1011D00003B0F0BDFC020020380300200003002013
:1011E000B000002074000020700000205C5F000848
:1011F0009C000020605F0008645F0008685F0008D2
:10120000FF0000106C5F00080000FF04680300206E
:10121000705F0008E8020020805F000800000020E6
:101220000400002085000020FFFFFF04F9000003F8
:10123000845F00082C2130004C0000209D0000201D
:1012400090B587B004AF7D4B1B78012B55D17C4BFB
:101250001A68DE235B42101C191C03F0ADFB784BAF
:101260001B68181C002103F0A7FB754B1968754A11
:10127000F3231B01081C111C1A1C03F0FBFA724B10
:10128000724A1A60C0466E4B1B68714A181C111CCA
:1012900003F0EEF9031C1C1C694B1B686D4A181CFB
:1012A000111C03F0E5F9031C9C42ECD1644B1B6854
:1012B000BC1D674A181C111C03F0DAF9031C2380BB
:1012C000654B00221A605E4B1B68181C002104F05D
:1012D00001FA5B4B1A68BB1D1B8860498C4663444E
:1012E000101C191C03F0E4F9021C5B4B1A605C4BE8
:1012F00000221A60514B00221A70514B1B68181CB7
:1013000004F05CFA4E4B1B68181C04F063F84C4B5D
:101310001B68544A181C111CFEF768FF484B1B68D9
:10132000514A181C111CFEF761FF454B1B684F4AC0
:10133000181C111CFEF75AFF414B1B684C4A181C25
:10134000111CFEF753FF3E4B1A6880235B04101CF0
:10135000191CFEF74BFF3A4B19683B4B1B681B7877
:101360001A1C1F231340DA04374B1B68DB689B05EC
:101370009B0D5B021A43344B1B689B68DB05DB0D3E
:101380001343E022D2041343081C191CFEF72EFF5E
:10139000384B96221A60384BB4221A60374BFA2227
:1013A0001A602F4B1A68131C5B009B189B001A1EB7
:1013B000324B1B689A420DDD214B19682F4B1B687D
:1013C000DB03DB0BA82252051343081C191CFEF794
:1013D0000DFF11E01A4B1968214B1A68131C5B00B2
:1013E0009B189B001A1C264B1340A822520513433E
:1013F000081C191CFEF7FAFE114B19681F4B1B68DD
:10140000DB03DB0BC82252051343081C191CFEF733
:10141000EDFE0B4B1A6880231B05101C191CFEF7F0
:10142000E5FE0F4B1B68DB00FF2B2DDD044B1B681B
:10143000144A181C111CFEF7D9FE34E0F8020020F3
:10144000FC02002000620008BC02002024000020F2
:10145000FC203000F8203000D8020020048030004A
:101460007C000020FFFFFF0207000026FFFFFF04B3
:101470000100001FF0020020B802002040030020FD
:10148000FCFF0100FF000010744B1968744B1B68CF
:10149000DB001A1CFF231340802252051343081C53
:1014A000191CFEF7A3FE6D4B19686E4B1B68DB051C
:1014B000DB0D5A056C4B1B68DB05DB0D1B0313436F
:1014C000802212061343081C191CFEF78FFE634B83
:1014D0001A6884239B05101C191CFEF787FE5F4BBE
:1014E0001B68624A181C111CFEF780FE5B4B1B68D0
:1014F0005F4A181C111CFEF779FE584B1B685D4AA9
:10150000181C111CFEF772FE544B1B685A4A181C1B
:10151000111CFEF76BFE594B00221A70574B181C1A
:1015200004F078FC031C1A1C544BD218544B111CA9
:101530001A1C0E23081C111C1A1C04F02DFC514B04
:101540001B68181C642104F0A5FA031C01331A1C43
:101550004A4B181C111C03F083FA484B181C04F06A
:1015600059FC031C1A1C454BD218474B111C1A1C62
:101570000223081C111C1A1C04F00EFC374B1868BF
:10158000424B1968424B1B680C3B1A1C80231B0101
:1015900000933A4B0193142303F06EFE3D4B1B78EE
:1015A000DBB2022B0ED03B4B1B78DBB2032B09D0F6
:1015B000384B1B78DBB2052B04D0364B1B78DBB2E3
:1015C000062B2DD1254B1B68334A181C111CFEF726
:1015D0000DFE224B1B68314A181C111CFEF706FE3B
:1015E0001E4B1868294B1B68413B191C284B1B6874
:1015F0002A3B1A1C1E2300931423019300230293F9
:10160000274B03933C2303F01DFF144B1B68254A13
:10161000181C111C03F00CF8031C1A1C224B1A7026
:101620000E4B1B68181C0021FEF7E0FD0B4B1B68DE
:10163000181C03F0B7FE094B1B68181CFEF7ECFDE5
:10164000064B1B68181C03F08FF9054B1B685A1CCE
:10165000034B1A60BD4603B090BDC046FC0200209B
:101660007C000020F0020020B802002000010015DC
:1016700000010019FF0000100000FF0468030020B3
:10168000705F0008E8020020805F00080000002072
:101690000400002085000020FFFFFF04F900000384
:1016A000845F00082C2130004C000020B0B588B0C9
:1016B00004AF2823FB601023BB60BA68131CDB0750
:1016C0009B1A5B001A1CF84B1B68D218F74B196861
:1016D000FB68C91ABB68CB1A53437B60F44B1B7879
:1016E000012B0CD1F34B1968F34B1A687B68081C6B
:1016F000111C1A1C03F0C8FFED4B00221A70EF4BAF
:101700001B78DBB2022B04D0EC4B1B78DBB2052B31
:1017100024D1E84B1868BB689BB21A1CD203D31AB9
:10172000DB189AB2E04B1B689BB2D3189CB2DF4B1C
:101730001B689AB2FB689BB2D31A9AB2BB689BB281
:10174000D31A9AB2DC4B1B68B968FD68009201930A
:10175000032302932A1C231C03F0C8FED74B1B78DB
:10176000DBB2032B04D0D54B1B78DBB2062B26D182
:10177000D04B1868BB689BB21A1CD203D31ADB1873
:101780009AB2C94B1B689BB2D3189CB2C74B1B685B
:101790009AB2FB689BB2D31A9AB2BB689BB2D31AB7
:1017A0009AB2C54B1B68B968FD6800920193032388
:1017B0000293C34B03932A1C231C03F0D9FEBD4B99
:1017C0001B68181C03F0FAFFBA4B1B68BD4A181CB3
:1017D000111CFEF70BFDB74B1B68BB4A181C111CF4
:1017E000FEF704FDB34B1B68B84A181C111CFEF72A
:1017F000FDFCB04B1868AC4B1B681B051B0D1A0396
:10180000AA4B1968FB68CB1A1B051B0D1343E0227A
:1018100052051343191CFEF7E9FCA64B1968FB6837
:101820005B055B0DD82252051343081C191CFEF7FB
:10183000DDFCA04B1B68A64A181C111CFEF7D6FC49
:101840009C4B1B68A04A181C111CFEF7CFFC994B3F
:101850001B689E4A181C111CFEF7C8FC954B1868A3
:10186000BA68131CDB079B1A5B001A1C8E4B1B68A3
:10187000D3181B051B0D1A038C4B1968FB68C91A7A
:10188000BB68CB1A1B051B0D1343E0225205134303
:10189000191CFEF7ABFC874B1968BB685B055B0D39
:1018A000DA02FB685B055B0D1343D8225205134334
:1018B000081C191CFEF79AFC7E4B1B68854A181CF5
:1018C000111CFEF793FC7B4B1B687F4A181C111CF4
:1018D000FEF78CFC774B1B687F4A181C111CFEF727
:1018E00085FC744B1A68D8235B05101C191CFEF785
:1018F0007DFC704B1A688023DB04101C191CFEF75A
:1019000075FC6C4B1B68754A181C111CFEF76EFCAD
:10191000684B1968684B1B689B029B0A8022520423
:101920001343081C191CFEF761FC624B1868BA6867
:10193000131CDB079B1A5B001A1C5B4B1B68D3183C
:101940009B059B0D5A02594B1968FB68C91ABB6865
:10195000CB1ADB05DB0D1343E322D2041343191C1E
:10196000FEF744FC534B1868FA68131CDB079B1AFC
:101970005B001A1C4C4B1B68D3189B121A1C0323C8
:1019800013409900FA68131CDB079B1A5B001A1CB2
:10199000464B1B68D3185B121A1C032313400B43DE
:1019A000A02292051343191CFEF720FC414B186836
:1019B000BA68131CDB079B1A5B001A1C3A4B1B68A6
:1019C000D318DB05DB0D5A02384B1968FB68C91ABE
:1019D000BB68CB1ADB05DB0D1343812212051343D1
:1019E000191CFEF703FC334B1868FA68131CDB075D
:1019F0009B1A5B001A1C2C4B1B68D3185B121A1C19
:101A0000032313409900FA68131CDB079B1A5B0041
:101A10001A1C264B1B68D3185B121A1C0323134095
:101A20000B43A42292051343191CFEF7DFFB214B45
:101A30001968BB681B011A1C294B1340DA03FB68A9
:101A40001B01181C264B034013438022D20513436D
:101A5000081C191CFEF7CAFB164B1A6884239B0549
:101A6000101C191CFEF7C2FB124B1B68174A181CEE
:101A7000111CFEF7BBFB0F4B1A680B4B1B68002BAE
:101A800000DA01335B10191CC023DB000093154BF7
:101A90000193101C14221B2303F0EEFB054B1B6863
:101AA000114A181C111C21E0000000200400002035
:101AB000F8020020FC020020D8020020850000204F
:101AC000DC050000FF00000207000026FFFFFF0406
:101AD000E0E0E002FFFFFF020008801C0100001FA1
:101AE000F07F00008C5F00080000FF04FEF77EFB23
:101AF000704B00221A706F4B181C04F08BF9031CFA
:101B00001A1C6C4BD2186C4B111C1A1C0E23081C8F
:101B1000111C1A1C04F040F9684B1B68181C642146
:101B200003F0B8FF031C01331A1C624B181C111C74
:101B300002F096FF5F4B181C04F06CF9031C1A1C92
:101B40005C4BD2185E4B111C1A1C0223081C111C82
:101B50001A1C04F021F95B4B18685B4B19685B4B4E
:101B60001B680C3B1A1C80231B010093514B0193F3
:101B7000142303F081FB564B1B78DBB2022B0ED0F3
:101B8000534B1B78DBB2032B09D0514B1B78DBB2D4
:101B9000052B04D04E4B1B78DBB2062B64D1494B8E
:101BA0001B684C4A181C111CFEF720FB454B1B6898
:101BB000494A181C111CFEF719FB424B1868424B8E
:101BC0001B68413B191C414B1B682A3B1A1C1E23F6
:101BD00000931423019300230293404B03933C236F
:101BE00003F030FC374B1B683D4A181C111C02F0F7
:101BF0001FFD031C1A1C3B4B1A70324B1B683A4AE0
:101C0000181C111CFEF7F2FA2E4B19682E4B1B689C
:101C1000413B1A1C1E2300931423019300230293BB
:101C2000324B0393081C111C0C223C2303F00AFCCA
:101C3000244B1B682A4A181C111C02F0F9FC031CD7
:101C40001A1C2B4B1A702A4B1B78FA2B0CD11D4BEC
:101C50001968284B1A687B68081C111C1A1C03F0B1
:101C600013FD234B00221A70164B1B68181C002111
:101C7000FEF7BCFA134B1B68181C03F093FB114BC7
:101C80001B68181CFEF7C8FA0E4B1B68181C02F0E4
:101C90006BFE0C4B1A68E9235B42101C191C02F006
:101CA0008BFE084B1B68181C02F05EFEBD4604B09C
:101CB000B0BDC04668030020705F0008E802002045
:101CC000805F0008FC0200200000002004000020CB
:101CD00085000020FFFFFF04F9000003845F000877
:101CE0002C2130004C000020FA000003985F00080F
:101CF0004D000020D802002080B500AF034B002229
:101D00001A60024B00225A71BD4680BD440000207B
:101D100090B587B000AF78603960314B1B68314AAD
:101D2000181C111C02F0C4FC031C7B612C4B1B68AB
:101D30002D4A181C111C02F0BBFC031C3B61284BF4
:101D40001B682A4A181C111C02F0B2FC031CFB6021
:101D5000234B1B68264A181C111C02F0A9FC031C0B
:101D6000BB607B691B0C1A1C7B681A607A693B6834
:101D70001A607B6804333A69120C1A603B680433BA
:101D80003A691A607B680833FA68120C1A603B687B
:101D90000833FA681A607B680C33BA68120C1A6050
:101DA0003B680C33BA681A607B6810331C1C0C4B00
:101DB0001B68104A181C111C02F05AFC031C2360FB
:101DC0003B6810331C1C064B1B680B4A181C111C6B
:101DD00002F04EFC031C2360BD4607B090BDC04618
:101DE000FC020020242130001C2130008C21300016
:101DF000902130006C2130002021300080B586B069
:101E000000AF786039601423FB1800221A807A68CA
:101E100080231B029A4202D17B6801337B603A68BF
:101E200080231B029A4202D13B6801333B603B682E
:101E30005A1E1343DB0FDAB27B68D917CB1ADB0FBC
:101E4000DBB25340DBB2002B0ED03B683B617B68BA
:101E50003B603B697B601423FB181422BA1812887C
:101E60008021C9014A401A803B68002B03DC3B6893
:101E70005B423B6007E01423FB181422BA18128857
:101E80002D494A401A807B68DA179B1853407B60C3
:101E90003A687B689A420DDD3B68FB607B683B607B
:101EA000FB687B601423FB181422BA18128823499C
:101EB0004A401A8005E03B685B103B607B685B1022
:101EC0007B603A687B6813431D4A1340F3D17B68FB
:101ED000002B04D11623FB1800221A801AE03A685E
:101EE0007B689A4205D11623FB18802292011A8042
:101EF00010E03B681B02181C796803F05BFE031CB2
:101F0000BB60BA680F4BD3181B789AB21623FB1824
:101F100052011A801623FB181622B9181422BA1877
:101F2000098812884A401A801623FB181B88181C3F
:101F3000BD4606B080BDC0460080FFFFFF3F0000E9
:101F400080FF0000A05F000880B500AF094B0022B1
:101F50001A70094BF02252011A60084B00221A60D5
:101F6000074B882252011A60064B00221A60BD46B8
:101F700080BDC0463D030020EC020020F40200209A
:101F8000DC0200204403002080B500AF1F4B00227C
:101F90001A701FE01E4B18681C4B1B781A1C1D4B37
:101FA0009200D3585B045B0CDA03184B1B78191CA6
:101FB000194B8900CB585B045B0C13438022D2057C
:101FC0001343191CFEF712F9104B1B780133DAB2D8
:101FD0000E4B1A700D4B1A78104B1B789A42D9D3BE
:101FE0000B4B19680B4B1B685B045B0CDA030A4B49
:101FF0001B685B045B0C13438022D2051343081C4F
:10200000191CFEF7F3F8BD4680BDC04684000020D1
:10201000FC02002018030020480300203D0300209C
:1020200080B500AFFFF790FF0B4B1A6880239B052C
:10203000101C191CFEF7DAF8074B1B68074A181C1E
:10204000111CFEF7D3F8044B1B68054A181C111C21
:10205000FEF7CCF8BD4680BDFC0200200D00000C50
:10206000FFFF070A80B582B000AF786039607B68F7
:102070001A111E4B1B689A4203DA7B681A111B4B1C
:102080001A607B681A111A4B1B689A4203DD7B6841
:102090001A11174B1A603B681A11164B1B689A42AB
:1020A00003DA3B681A11134B1A603B681A11124B82
:1020B0001B689A4203DD3B681A110F4B1A600F4BE5
:1020C0001B781A1C0E4B92007968D1500B4B1B7871
:1020D0001A1C0C4B92003968D150084B1B78013305
:1020E000DAB2064B1A70BD4602B080BDEC02002089
:1020F000F4020020DC020020440300203D03002005
:10210000180300204803002080B500AF054B1B6872
:10211000054A181C111CFEF769F8FFF735FFBD468C
:1021200080BDC046FC0200200400001F90B59DB099
:1021300004AF3023FB1802221A702F23FB1802224F
:102140001A70FEF7DFFBFEF731FC02F055F802F0E3
:10215000B7F8F34BF34A1A60012002F04BFC002061
:1021600002F014FB642002F0F5FC482002F00EFBA4
:102170000A2002F0EFFC9023DB05181C102100223E
:1021800002F0CCFF422002F0F3FC002002F0F0FC51
:10219000002002F0EDFC9023DB05181C1021012229
:1021A00002F0BCFF0A2002F0D5FC9023DB05181CCE
:1021B0001021002202F0B2FF612002F0D9FC0220BF
:1021C00002F0D6FC002002F0D3FC9023DB05181CA3
:1021D0001021012202F0A2FF142002F0BBFC00201B
:1021E00002F0D4FA642002F0B5FC5F23FB18002251
:1021F0001A70CB4B1B685F22BC18CB4A181C111CF1
:1022000002F016FA031C23700AE0C54B1B685F221C
:10221000BC18C54A181C111C02F00AFA031C2370D2
:102220005F23FB181B787C2BEFD1C8239B00BB6579
:10223000F0235B007B658423DB003B652E23FB647E
:102240000023BB640A237B64B84B3B641723FB6306
:102250000023BB630A237B633323FB1801221A701C
:102260003223FB1800221A703123FB1800221A7047
:10227000AB4B1A683B6D9BB2AD49101C1A1C02F0A7
:102280004FFAA74B1A68FB6C9BB2AA49101C1A1C88
:1022900002F046FAA24B1A68BB6C9BB2A649101C0E
:1022A0001A1C02F03DFA9E4B1A687B6C9BB2A34944
:1022B000101C1A1C02F034FA994B1A683B6C9BB242
:1022C0009F49101C1A1C02F02BFA954B1A68FB6BE5
:1022D0009BB29C49101C1A1C02F022FA904B1A68FF
:1022E000BB6B9BB29849101C1A1C02F019FA8C4B5C
:1022F0001A687B6B9BB29549101C1A1C02F010FAED
:10230000874B1A6892493223FB181B78101C1A1C41
:1023100002F0EAF9824B1B688E4A181C111C00223D
:1023200002F0E2F97E4B1A688B493123FB181B78C7
:10233000101C1A1C02F0D8F9794B1A68874933230C
:10234000FB181B78101C1A1C02F0CEF9744B1A688B
:10235000BB6D9BB28249101C1A1C02F0E1F9704B54
:102360001A687B6D9BB27F49101C1A1C02F0D8F9C9
:102370006B4B1C686A4B1B687B4A181C111C02F0D3
:1023800057F9031C1A1C7D235B421343DBB2764AC8
:10239000201C111C1A1C02F0A7F9614B1C68604B31
:1023A0001B68724A181C111C02F042F9031C1A1C0B
:1023B0007D235B421343DBB26C4A201C111C1A1CA8
:1023C00002F092F9564B1A6869499623DB00101CFB
:1023D0001A1C02F0A5F98023DB02181C0121FDF76D
:1023E0008DFE3B1C04221A603B1C01221A713B1C0F
:1023F00000229A713B1C03225A713B1C0022DA71A5
:102400005C4A3B1C101C191C02F0BAFDFDF710FFC2
:10241000594B5A4A1A60584B1B68181C002101225C
:10242000FEF73EF9554B1B78013BDAB2544B1A705C
:10243000544B01221A70544B00221A70534B012244
:102440001A70374B1B685249524A181C02F084F923
:10245000334B1B684E4A181C111C02F029F9031C4F
:10246000BB62484B1B78DBB2002B00D1A2E2454B8C
:1024700000221A70FFF740FC434B00221A70404BB9
:102480001B78DBB20133DBB23D4A191C1170072BFC
:1024900002D13B4B01221A70394B1B78DAB2374B11
:1024A0001A700020FDF786FF334B1B68181C0021B3
:1024B0000122FDF7E9FF384B01225A71304B1B789E
:1024C000DBB2062B00D941E19A00344BD3181B68CC
:1024D0009F46334B334A1A60C8239B00BB65F023E9
:1024E0005B007B658423DB003B652E23FB640023BC
:1024F000BB640A237B640D4B3B641723FB630023FF
:10250000BB630A237B633323FB1801221A70322337
:10251000FB1800221A703123FB1800221A7016E1F2
:10252000FC02002088000020002030000D02000086
:102530002C20300030203000382030003C2030008B
:1025400040203000442030004C203000502030002B
:1025500064203000682030006C2030007020300093
:10256000342030004820300090203000942030008B
:102570001821300000040048E4020020C0020020BE
:1025800085000020F90200204C0000208600002079
:102590000C2030000051250244000020A4610008F6
:1025A000A00000207C5E0008614B624A1A60C823CC
:1025B0009B00BB65F0235B007B658423DB003B65F0
:1025C0002E23FB640023BB640A237B645A4B3B64C9
:1025D0001723FB630023BB630A237B633323FB18AE
:1025E00001221A703223FB1800221A703123FB18C3
:1025F00000221A70ABE04E4B504A1A60C8239B0071
:10260000BB65F0235B007B658423DB003B652E23E9
:10261000FB640023BB640A237B64474B3B641723A2
:10262000FB630023BB630A237B633323FB18012274
:102630001A703223FB1800221A703123FB18002273
:102640001A7084E03A4B3E4A1A60C8239B00BB656F
:10265000F0235B007B658423DB003B652E23FB645A
:102660000023BB640A237B64334B3B641723FB6367
:102670000023BB630A237B633323FB1801221A70F8
:102680003223FB1800221A703123FB1800221A7023
:102690005DE0274B2B4A1A60C8239B00BB65F023E3
:1026A0005B007B658423DB003B652E23FB640023FA
:1026B000BB640A237B64204B3B641723FB6300232A
:1026C000BB630A237B633323FB1801221A70322376
:1026D000FB1800221A703123FB1800221A7036E012
:1026E000134B194A1A60C8239B00BB65F0235B009B
:1026F0007B658423DB003B652E23FB640023BB64E6
:102700000A237B640C4B3B641723FB630023BB63EE
:102710000A237B633323FB1801221A703223FB1830
:1027200000221A703123FB1800221A700FE0C046F5
:10273000A00000209C5E00080D020000BC5E0008A6
:10274000DC5E0008FC5E00081C5F0008C046E34B2E
:102750001A683B6D9BB2E249101C1A1C01F0E0FFA5
:10276000DE4B1A68FB6C9BB2DE49101C1A1C01F090
:10277000D7FFDA4B1A68BB6C9BB2DB49101C1A1CE2
:1027800001F0CEFFD54B1A687B6C9BB2D749101C69
:102790001A1C01F0C5FFD14B1A683B6C9BB2D4499F
:1027A000101C1A1C01F0BCFFCC4B1A68FB6B9BB2CF
:1027B000D049101C1A1C01F0B3FFC84B1A68BB6B40
:1027C0009BB2CD49101C1A1C01F0AAFFC34B1A681A
:1027D0007B6B9BB2C949101C1A1C01F0A1FFBF4BB7
:1027E0001A68C7493223FB181B78101C1A1C01F009
:1027F0007BFFBA4B1A68C3493123FB181B78101CA6
:102800001A1C01F071FFB54B1B68BF4A181C111C44
:10281000002201F069FFB14B1A68BC493323FB1851
:102820001B78101C1A1C01F05FFFAC4B1A68BB6DC3
:102830009BB2B749101C1A1C01F072FFA74B1A6813
:102840007B6D9BB2B349101C1A1C01F069FFA34BAE
:102850001C68A24B1B68B04A181C111C01F0E8FE52
:10286000031C1A1C7D235B421343DBB2AA4A201CC3
:10287000111C1A1C01F038FF984B1C68974B1B6801
:10288000A64A181C111C01F0D3FE031C1A1C7D2340
:102890005B421343DBB2A14A201C111C1A1C01F03D
:1028A00023FF8E4B1A689E499623DB00101C1A1CCE
:1028B00001F036FF894B1B689A4A181C111C002234
:1028C00001F012FF984B1B78DBB2032B2FD1834B07
:1028D0001B689649964A181C01F03EFF7F4B1B6807
:1028E000944A181C111C002201F036FF7B4B1B6818
:1028F000914A181C111C002201F02EFF774B1B6817
:102900008E4A181C111C002201F026FF734B1A6816
:102910008B49F023DB01101C1A1C01F01DFF6F4BCB
:102920001B68884A181C111C002201F015FF7E4B01
:102930001B78DBB2062B31D1684B1A687B498023A8
:102940005B02101C1A1C01F007FF644B1B68794ADC
:10295000181C111C002201F0FFFE604B1B68764A18
:10296000181C111C002201F0F7FE5C4B1B68734A17
:10297000181C111C002201F0EFFE584B1A68704918
:1029800080235B02101C1A1C01F0E6FE534B1B68EF
:102990006C4A181C111C002201F0DEFE6A4B00225A
:1029A0001A706A4B1A68684B1B789B00D3181A6818
:1029B000674B1A60644B1B78082B00D951E59A00CD
:1029C000644BD3181B689F46444B1B68181C02F0CD
:1029D000F5FE424B1B68604A181C111CFDF706FCF3
:1029E0003E4B1B685D4A181C111CFDF7FFFB3B4B5F
:1029F0001A689023DB04101C191CFDF7F7FB4A4BE7
:102A00001B78DBB2062B00D9E6E09A00544BD318B2
:102A10001B689F46314B1A68BB6D002B00DA0133EF
:102A20005B10191C7B6D002B00DA01335B101C1C42
:102A300080239B0000934B4B0193101C221C1C23F2
:102A400002F01AFCC8E0254B1A68BB6D002B00DAB7
:102A500001335B10191C7B6D002B00DA01335B1016
:102A60001C1C80239B0000933F4B0193101C221CD5
:102A70001C2302F001FCAFE0184B1A68BB6D002B61
:102A800000DA01335B10191C7B6D002B00DA013377
:102A90005B101C1C80239B000093344B0193101C83
:102AA000221C1C2302F0E8FB96E00C4B1A68BB6D5D
:102AB000002B00DA01335B10191C7B6D002B00DA50
:102AC00001335B101C1C80239B000093284B019357
:102AD000101C221C1C2302F0CFFB7DE0FC02002016
:102AE0002C20300030203000382030003C203000D6
:102AF00040203000442030004C2030005020300076
:102B0000642030006C2030006820300070203000DD
:102B100034203000482030009020300094203000D5
:102B2000182130005820300085000020502130004E
:102B3000DA72000054213000582130005C2130004E
:102B4000602130006421300078000020A0000020C7
:102B5000E8020020C0610008FFFFFF020700002616
:102B6000E4610008A0600008BC600008D4600008B0
:102B7000EC600008CF4B1A68BB6D002B00DA013304
:102B80005B10191C7B6D002B00DA01335B101C1CE1
:102B900080239B000093C84B0193101C221C1C2314
:102BA00002F06AFB18E0C34B1A68BB6D002B00DA19
:102BB00001335B10191C7B6D002B00DA01335B10B5
:102BC0001C1C80239B000093BC4B0193101C221CF7
:102BD0001C2302F051FBC046B64B1B68B84A181CB8
:102BE000111CFDF703FBB74B00221A70B54B181CE4
:102BF00003F010F9031C1A1CB24BD218B24B111C73
:102C00001A1C0E23081C111C1A1C03F0C5F8AF4B2C
:102C10001B68181C642102F03DFF031C01331A1CC1
:102C2000A84B181C111C01F01BFFA64B181C03F02D
:102C3000F1F8031C1A1CA34BD218A54B111C1A1C2B
:102C40000223081C111C1A1C03F0A6F8994B1868E3
:102C50007B6D0C3B1A1CB96D80231B010093994BB3
:102C60000193142302F008FB9A4B1B78DBB2032B71
:102C700004D0984B1B78DBB2062B2BD18D4B1B68F5
:102C8000954A181C111CFDF7B1FA8A4B1B68934A30
:102C9000181C111CFDF7AAFA864B1868BB6D413B46
:102CA000191C7B6D2A3B1A1C1E23009314230193CD
:102CB000002302938A4B03933C2302F0C3FB7D4B1A
:102CC0001B68884A181C111C01F0B2FC031C1A1C5A
:102CD000854B1A707F4B1B78DBB2022B04D07D4BE7
:102CE0001B78DBB2052B2FD1804B1B78002B2BD10F
:102CF000704B1B68784A181C111CFDF777FA6D4B56
:102D00001B68764A181C111CFDF770FA694B18688D
:102D1000BB6D413B191C7B6D2A3B1A1C1E23009383
:102D200014230193002302936D4B03933C2302F081
:102D300089FB604B1B686B4A181C111C01F078FC66
:102D4000031C1A1C684B1A705A4B1B68181C002174
:102D5000FDF74CFA574B1B68181C02F023FB554B30
:102D60001B68181CFDF758FA524B1B68181C01F021
:102D7000FBFD01F094F85E4B1B78012B00D095E031
:102D80005A4B1B78012B00D090E0524B1B78DBB2E2
:102D9000022B05D04F4B1B78DBB2052B00D085E012
:102DA000544B00225A71434B1B68181C02F006FD5D
:102DB000404B1A6880239B04101C191CFDF716FA5F
:102DC0003C4B1B684C4A181C111CFDF70FFA394B81
:102DD0001B68414A181C111CFDF708FA354B1A688C
:102DE000BB6D002B00DA01335B10191C7B6D002BCF
:102DF00000DA01335B101C1CC023DB0000933F4B47
:102E00000193101C221C1B2302F036FA294B1B686D
:102E1000181C002102F014FC264B1B68181C002112
:102E2000FDF7E4F9234B1B68181C02F0BBFA214B99
:102E30001B68181CFDF7F0F91E4B1B68181C01F0ED
:102E400093FD2A4B00221A702A4B01225A71194B0A
:102E50001B68181C02F0B2FC164B1B68284A181C91
:102E6000111CFDF7C3F9134B1B68234A181C111CD6
:102E7000FDF7BCF90F4B1B68174A181C111CFDF716
:102E8000B5F90C4B1B68181C0021FDF7AFF9094B75
:102E90001B68181C02F086FA064B1B68181CFDF70D
:102EA000BBF9044B1B68181C01F05EFDFEF7C8F966
:102EB00000F0F5FFFC020020086100082061000816
:102EC0000000FF0468030020705F0008E802002093
:102ED000805F000885000020FFFFFF04F900000369
:102EE000845F00082C2130004C0000208600002068
:102EF000F802002044000020070000263861000886
:102F0000FFFFFF02C04B1B68C04A181C111C0122A6
:102F100001F0EAFBBE4B1B78DBB2022B0ED0BC4BA0
:102F20001B78DBB2032B09D0B94B1B78DBB2052B26
:102F300004D0B74B1B78DBB2062B39D1B24B1B68E0
:102F4000B44A181C111C01F0B3FB031C7B62AE4B8E
:102F50001B68B14A181C111C01F0AAFB031C3B6240
:102F6000A94B1B68AD4A181C111C01F0A1FB031CE6
:102F7000FB61A54B1B68AA4A181C111C01F098FBA9
:102F8000031CBB61A04B1B68A64A181C111C01F056
:102F90008FFB031C7B619C4B1B68A34A181C111CF4
:102FA00001F086FB031C3B61FEF780FB00F077FF1E
:102FB00000F075FF944B1B68944A181C111C0022EA
:102FC00001F092FB904B1B68984A181C111CFDF7EE
:102FD0000DF98D4B1B68964A181C111CFDF706F95C
:102FE000894B1B68934A181C111CFDF7FFF8864B90
:102FF0001A6888239B05101C191CFDF7F7F8824BF3
:103000001B688D4A181C111CFDF7F0F87E4B1A68DE
:10301000BB6D002B00DA01335B10191C7B6D002B9C
:1030200000DA01335B101C1CC023DB000093834BD0
:103030000193101C221C1B2302F01EF9724B1B680B
:103040007F4A181C111CFDF7D1F87E4B00221A7024
:103050007C4B181C02F0DEFE031C1A1C794BD218A4
:10306000794B111C1A1C0E23081C111C1A1C02F08F
:1030700093FE764B1B68181C642102F00BFD031CA9
:1030800001331A1C6F4B181C111C01F0E9FC6D4B2D
:10309000181C02F0BFFE031C1A1C6A4BD2186C4BA2
:1030A000111C1A1C0223081C111C1A1C02F074FEAD
:1030B000554B18687B6D0C3B1A1CB96D80231B01A6
:1030C0000093604B0193142302F0D6F84E4B1B681B
:1030D000604A181C111CFDF789F84B4B1B68181C23
:1030E00001F042FC5C4A5D4B101C191CFEF710FEFF
:1030F0005B4B00221A605B4B00221A605A4B002285
:103100001A705A4B00221A6027E0584B1A68524B2B
:103110009200D25880231B029A4219D0534B1A684E
:103120004D4B9200D2584E4B1B68D2184C4B1A6034
:103130004E4B1A68494B9200D2584A4B1B68D21822
:10314000484B1A60484B1B780133DAB2464B1A7071
:10315000464B1B685A1C454B1A60444B1B68042B9A
:10316000D3DD414B1B78002B17D03D4B1A683E4BEB
:103170001B78101C191C02F01DFD031C1A1C384B77
:103180001A60384B1A68384B1B78101C191C02F057
:1031900011FD031C1A1C334B1A60334B1B78002B98
:1031A00028D0324B00221A6020E0304B1C682F4B95
:1031B0001A68294B9200D258294B1B68D11A2B4B05
:1031C0001A68264B9200D258264B1B68D31A081C4B
:1031D000191CFEF713FE031C1B0A9BB2DAB2244B28
:1031E0001A55224B1B685A1C204B1A601F4B1B6838
:1031F000042BDADDFEF714FF1E4B00221A606BE091
:103200001A4B00221A605EE0FC0200200821300008
:10321000850000205021300054213000582130001A
:103220005C213000602130006421300000FFFFFF8E
:103230005000000207000026FFFFFF045061000855
:103240000000FF0468030020705F0008E80200200F
:10325000805F000840404004C402002004030020B6
:103260005C0000206000002064000020500000206E
:10327000A4000020540000206C4B1B686C4AD35CF7
:103280001A1E6C4B1B689A4218D1684B1A686A4B1D
:103290009200D25880231B029A420FD0634B1A68C7
:1032A000654B9200D3581901604B1A68634B92002A
:1032B000D3581B01081C191CFEF7D4FE5B4B1B687E
:1032C0005A1C5A4B1A60594B1B68042BD4DD594BBE
:1032D0001B685A1C574B1A60564B1B68FF2B8FDD1F
:1032E000574B1B68574A181C111CFCF77FFF544BA7
:1032F0001B68554A181C111CFCF778FF504B1B68C3
:10330000524A181C111CFCF771FF4D4B1B68504AA8
:10331000181C111CFCF76AFF494B1B684D4A181C0E
:10332000111CFCF763FF464B1A6880231B06101C18
:10333000191CFCF75BFF424B1B68474A181C111C09
:10334000FCF754FF3E4B1A688C239B05101C191C7C
:10335000FCF74CFF3A4B1B68404A181C111CFCF749
:1033600045FF374B1B683E4A181C111CFCF73EFFFB
:10337000FEF7CAFE3B4B1B78DBB2022B0ED0394B5B
:103380001B78DBB2032B09D0364B1B78DBB2052B45
:1033900004D0344B1B78DBB2062B2BD1284B1B6897
:1033A000314A181C111CFCF721FF254B1B682F4AC2
:1033B000181C111CFCF71AFF214B1868BB6D413B10
:1033C000191C7B6D2A3B1A1C1E23009314230193A6
:1033D00000230293264B03933C2302F033F8184B4F
:1033E0001B68244A181C111C01F022F9031C1A1C2A
:1033F000214B1A70124B1B68181C0021FCF7F6FEBB
:103400000F4B1B68181C01F0CDFF0D4B1B68181CDF
:1034100001F07CFF0A4B1B68181CFCF7FDFE00F056
:103420003EFDFDF79FFB00F03AFDC0465000002036
:10343000A400002054000020C40200200403002047
:10344000FC020020FF0000100F0000201100000B04
:10345000FFFF050A0900001F000011BCFF80800467
:103460001800000E85000020FFFFFF04F900000394
:10347000845F00082C2130004C0000207B6D313B24
:10348000FB60BB6D002B00DA01335B10BB60DC4BD3
:103490001B68181C02F092F9D94B1B68D94A181CFA
:1034A000111CFCF7A3FED64B1B68D74A181C111C35
:1034B000FCF79CFED24B1A689023DB04101C191CED
:1034C000FCF794FECE4B1C68BB6D181C052102F066
:1034D00071FB031C1B011A1CCC4B1340D02212059C
:1034E0001343201C191CFCF781FEC54B1B68C84AFE
:1034F000181C111CFCF77AFEC14B1C68BB6D181C14
:10350000052102F057FB031C1B011A1CC14B134081
:10351000DA037B6D002B00DA01335B101B01191CF1
:10352000BC4B0B4013438022D2051343201C191CB3
:10353000FCF75CFEB24B1B68B74A181C111CFCF769
:1035400055FEAF4B1C68BB6D181C062102F032FB08
:10355000031C1B011A1CAD4B1340D0221205134350
:10356000201C191CFCF742FEA54B1C68BB6D5B00C0
:10357000181C052102F01EFB031C1B011A1CA54B85
:103580001340DA037B6D002B00DA01335B101B0163
:10359000191CA04B0B4013438022D2051343201C5F
:1035A000191CFCF723FE964B1B689C4A181C111C27
:1035B000FCF71CFE924B1C68BB6D181C072102F027
:1035C000F9FA031C1B011A1C904B1340D022120560
:1035D0001343201C191CFCF709FE894B1C68BA6DAB
:1035E000131C5B009B18181C052102F0E3FA031C56
:1035F0001B011A1C874B1340DA037B6D002B00DA8A
:1036000001335B101B01191C824B0B4013438022BA
:10361000D2051343201C191CFCF7E8FD784B1B68EE
:103620007F4A181C111CFCF7E1FD754B1968BB6D36
:10363000002B00DA0733DB101B011A1C734B1340FD
:10364000D02212051343081C191CFCF7CFFD6C4B4C
:103650001C68BB6D9B00181C052102F0ABFA031C13
:103660001B011A1C6B4B1340DA037B6D002B00DA35
:1036700001335B101B01191C664B0B401343802266
:10368000D2051343201C191CFCF7B0FD5C4B1B68D2
:10369000644A181C111CFCF7A9FD594B1A688423B5
:1036A0009B05101C191CFCF7A1FD554B1868B96847
:1036B000FA6880239B0000935B4B01931F2301F06A
:1036C000DBFD4F4B1B68594A181C111CFCF78EFD83
:1036D000574B00221A70564B181C02F09BFB031C20
:1036E0001A1C534BD218534B111C1A1C0E23081CC6
:1036F000111C1A1C02F050FB4F4B1B68181C642154
:1037000002F0C8F9031C01331A1C494B181C111C88
:1037100001F0A6F9464B181C02F07CFB031C1A1C96
:10372000434BD218454B111C1A1C0223081C111CB8
:103730001A1C02F031FB324B18687B6D0C3B1A1CD3
:10374000B96D80231B010093394B0193142301F0C1
:1037500093FD3B4B1B78DBB2022B0ED0384B1B7812
:10376000DBB2032B09D0364B1B78DBB2052B04D020
:10377000334B1B78DBB2062B2BD1214B1B68314A14
:10378000181C111CFCF732FD1D4B1B682E4A181C1F
:10379000111CFCF72BFD1A4B1868BB6D413B191C23
:1037A0007B6D2A3B1A1C1E230093142301930023D4
:1037B0000293264B03933C2301F044FE104B1B68FD
:1037C000234A181C111C00F033FF031C1A1C214B48
:1037D0001A700B4B1B68181C0021FCF707FD084BE7
:1037E0001B68181C01F0DEFD054B1B68181CFCF75C
:1037F00013FD034B1B68181C01F0B6F84FE3C046DD
:10380000FC020020FFFFFF0207000026F01F00005F
:103810000200001FF07F0000008000048000000410
:103820000080800480800004706100080000FF04B4
:1038300068030020705F0008E8020020805F000835
:1038400085000020FFFFFF04F9000003845F0008EB
:103850002C2130004C000020D64B1B68181C01F0B6
:10386000ADFFD44B1A6880239B04101C191CFCF775
:10387000BDFCD04B1B68D04A181C111CFCF7B6FCD1
:10388000CC4B1B68CD4A181C111CFCF7AFFCC94B74
:103890001A68BB6D002B00DA01335B10191CC023C2
:1038A000DB000093C64B0193101C14221B2301F074
:1038B000E3FCC04B1A68BB6D002B00DA01335B10D0
:1038C000191CC023DB000093BE4B0193101C3C224B
:1038D0001B2301F0D1FCB74B1B68BB4A181C111C01
:1038E000FCF784FCB94B00221A70B84B181C02F08C
:1038F00091FA031C1A1CB54BD218B54B111C1A1C9B
:103900000E23081C111C1A1C02F046FAB14B1B684E
:10391000181C642102F0BEF8031C01331A1CAB4BC7
:10392000181C111C01F09CF8A84B181C02F072FA2C
:10393000031C1A1CA54BD218A74B111C1A1C0223DE
:10394000081C111C1A1C02F027FA9A4B18687B6D90
:103950000C3B1A1CB96D80231B0100939B4B0193F8
:10396000142301F089FC9D4B1B78DBB2022B0ED097
:103970009A4B1B78DBB2032B09D0984B1B78DBB238
:10398000052B04D0954B1B78DBB2062B33D1894B2A
:103990001B688A4A181C111CFCF728FC854B1B6805
:1039A0008F4A181C111CFCF721FC824B1868BB6D58
:1039B000413B191C7B6D2A3B1A1C1E2300931423C8
:1039C000019300230293874B03933C2301F03AFDBC
:1039D000784B1B68844A181C111C00F029FE031C3C
:1039E0001A1C824B1A70734B1A68A0235B05101CBB
:1039F000191CFCF7FBFB6F4B1B68704A181C111C51
:103A0000FCF7F4FB6B4B1B68181C01F0E3FC784BD4
:103A10001A68784B1B789B00D3181B689A08131CF4
:103A20005B009A186B4B1B689A4214D2614B1A6860
:103A3000BB6D002B00DA01335B10191C7B6D002B72
:103A400000DA01335B101C1C00230093101C221CA5
:103A5000002301F073FC664B1A68664B1B789B00D1
:103A6000D3181B689A08131C5B009A18594B1B68E3
:103A70009A4220D35E4B1A685E4B1B789B00D3188A
:103A80001B685A08534B1B689A4214D2494B1A6858
:103A9000BB6D002B00DA01335B10191C7B6D002B12
:103AA00000DA01335B101C1C00230093101C221C45
:103AB000012301F043FC4E4B1A684E4B1B789B00D0
:103AC000D3181B685A08434B1B689A4220D3484BB3
:103AD0001A68484B1B789B00D3181B689A083D4B0B
:103AE0001B689A4214D2334B1A68BB6D002B00DA64
:103AF00001335B10191C7B6D002B00DA01335B1066
:103B00001C1C00230093101C221C022301F016FC35
:103B1000374B1A68374B1B789B00D3181B689A08E1
:103B20002C4B1B689A4214D3224B1A68BB6D002B96
:103B300000DA01335B10191C7B6D002B00DA0133B6
:103B40005B101C1C00230093101C221C032301F09B
:103B5000F5FB224B1B78DBB2022B0ED01F4B1B78E0
:103B6000DBB2032B09D01D4B1B78DBB2052B04D035
:103B70001A4B1B78DBB2062B06D10E4B1B681E4A74
:103B8000181C111CFCF732FB0A4B1B68181C002187
:103B9000FCF72CFB074B1B68181C01F003FC054BC2
:103BA0001B68181CFCF738FB024B1B68181C00F044
:103BB000DBFE74E1FC02002007000026FFFFFF048B
:103BC00078610008946100080000FF046803002089
:103BD000705F0008E8020020805F00088500002078
:103BE000F9000003845F00082C2130004C00002005
:103BF000A00000207800002001000014A94B1B68E1
:103C0000181C01F0DBFDA74B1B68A74A181C111CF0
:103C1000FCF7ECFAA34B1B68A44A181C111CFCF718
:103C2000E5FAA04B1B68A24A181C111CFCF7DEFA2F
:103C30009C4B1B689F4A181C111CFCF7D7FAFCF719
:103C4000C5FE984B1B689C4A181C111CFCF7CEFA49
:103C5000944B1B68994A181C111CFCF7C7FAFCF717
:103C6000B5FE904B1A688023DB04101C191CFCF76E
:103C7000BDFA8C4B1B68924A181C111CFCF7B6FA53
:103C8000884B1B688F4A181C111CFCF7AFFA854B38
:103C90001B688D4A181C111CFCF7A8FA814B1B6885
:103CA0008A4A181C111CFCF7A1FA7E4B1B68884A33
:103CB000181C111CFCF79AFA7A4B1B68854A181CD1
:103CC000111CFCF793FA774B1B68834A181C111CD4
:103CD000FCF78CFA734B1A6884239B05101C191C83
:103CE000FCF784FA6F4B1B687C4A181C111CFCF70C
:103CF0007DFA7B4B00221A70794B181C02F08AF86F
:103D0000031C1A1C764BD218764B111C1A1C0E235E
:103D1000081C111C1A1C02F03FF8734B1B68181C7E
:103D2000642101F0B7FE031C01331A1C6C4B181CF4
:103D3000111C00F095FE6A4B181C02F06BF8031C76
:103D40001A1C674BD218694B111C1A1C0223081C41
:103D5000111C1A1C02F020F8524B18687B6D0C3BAA
:103D60001A1CB96D80231B0100935D4B0193142332
:103D700001F082FA5E4B1B78DBB2022B0ED05C4B5B
:103D80001B78DBB2032B09D0594B1B78DBB2052B18
:103D900004D0574B1B78DBB2062B2BD1414B1B6851
:103DA000544A181C111CFCF721FA3E4B1B68524A5E
:103DB000181C111CFCF71AFA3A4B1868BB6D413BF2
:103DC000191C7B6D2A3B1A1C1E230093142301939C
:103DD00000230293494B03933C2301F033FB314B07
:103DE0001B68474A181C111C00F022FC031C1A1CFB
:103DF000444B1A702B4B1B68181C0021FCF7F6F97A
:103E0000284B1B68181C01F0CDFA264B1B68181CA8
:103E1000FCF702FA234B1B68181C00F0A5FD3EE0DE
:103E2000204B1B68181C01F0C9FC1E4B1B68364A4E
:103E3000181C111CFCF7DAF91A4B1B681B4A181CDA
:103E4000111CFCF7D3F9174B1B68181C0021FCF759
:103E5000CDF9144B1B68181C01F0A4FA114B1B6818
:103E6000181CFCF7D9F90F4B1B68181C00F07CFDDF
:103E7000264B01221A701E4B1B78DBB2013BDAB2D3
:103E80001B4B1A70224B00221A70224B1A68204BCF
:103E90001B789B00D3181A68134B1A60C046FEF7B4
:103EA000E0FAC046FC020020E0E8EC020700002631
:103EB000889DAA043F00000EFAFAFA043000000EB2
:103EC0000100001FCDBD059EE1BD859FE9BD85A018
:103ED000EEBDE5A0F3BD65A2AEBDC5A30000FF0425
:103EE00068030020705F0008E8020020805F00087F
:103EF00085000020FFFFFF04F9000003845F000835
:103F00002C2130004C000020FFFFFF02F9020020AE
:103F100078000020A000002080B500AF022001F052
:103F2000D7FC031E05D0044B01221A70022001F0B9
:103F3000EFFCBD4680BDC046A900002080B500AFA3
:103F4000504B5B79012B00D075E04E4B1B685A1C1F
:103F50004C4B1A604B4B1B68181C0A2101F020FEC9
:103F60000B1E68D1484B1B685A1E474B1A60464BC4
:103F70001B68002B25D1454B1B780133DAB2434B2C
:103F80001A70434B1A68414B1B789B00D3181A6870
:103F90003D4B1A600EE03D4B1B780133DAB23B4BD0
:103FA0001A703B4B1A68394B1B789B00D3181A6860
:103FB000354B1A60344B1B68002BECD0354B01227B
:103FC0001A70354B1B78F92B35D1314B1A682F4BB2
:103FD0001B789B00D3181B68323B1A1E2A4B1B68A8
:103FE0009A4228D92C4B00221A70284B1B78013397
:103FF000DAB2264B1A70264B1A68244B1B789B00AA
:10400000D3181A68204B1A600EE0204B1B7801333E
:10401000DAB21E4B1A701E4B1A681C4B1B789B00A1
:10402000D3181A68184B1A60174B1B68002BECD07A
:10403000184B01221A70194B1B78DBB2002B1ED0D3
:10404000174B1B78DBB20133DAB2154B1A70144BE5
:104050001B78DBB2052B12D1114B00221A70114BC9
:10406000181C022101F036F8031E05D10E4B012267
:104070001A700E4B01221A70084B00221A70BD46AE
:1040800080BDC04644000020E802002078000020E7
:10409000A0000020F80200204C000020A900002011
:1040A0004100002000040048F902002086000020A2
:1040B00080B500AF3A4A80239B01101C191C00F008
:1040C000CBFE031E0DD0364A80239B01101C191C09
:1040D00000F006FF334B1B78DBB20133DAB2314B11
:1040E0001A702F4A80235B01101C191C00F0B4FECB
:1040F000031E06D02A4A80235B01101C191C00F005
:10410000EFFE274A80239B00101C191C00F0A4FE20
:10411000031E06D0224A80239B00101C191C00F0AD
:10412000DFFE1F4A80231B01101C191C00F094FEA7
:10413000031E06D01A4A80231B01101C191C00F014
:10414000CFFE174A8023DB00101C191C00F084FEF0
:10415000031E06D0124A8023DB00101C191C00F03D
:10416000BFFE0F4B181C102100F076FE031E04D07A
:104170000B4B181C102100F0B3FE094A80235B0092
:10418000101C191C00F068FE031E06D0044A802390
:104190005B00101C191C00F0A3FEBD4680BDC0468C
:1041A000005400403C0300200C488546002103E0F9
:1041B0000B4B5B58435004310A480B4B42189A4250
:1041C000F6D30A4A02E0002313600432084B9A42F5
:1041D000F9D300F091FEFDF7A9FFFEE700100020E3
:1041E000247C000800000020380000203800002057
:1041F0007C030020FEE7000080B582B000AF3B1CCE
:10420000181C00F04FFF80239B02181C0121FBF7B4
:1042100075FF3B1C10221A603B1C01221A713B1CCB
:1042200003225A713B1C00229A713B1C0022DA7156
:104230009023DA053B1C101C191C00F0A1FE3B1C4E
:1042400004221A603B1C01221A713B1C03225A7182
:104250003B1C00229A713B1C0022DA719023DA0584
:104260003B1C101C191C00F08BFE3B1C181C00F0A2
:1042700019FF3B1C02221A603B1C00221A713B1CD6
:1042800003225A713B1C0122DA719023DA053B1C90
:10429000101C191C00F074FE9023DB05181C04216F
:1042A000012200F03BFF9023DB05181C10210122A6
:1042B00000F034FF0123181CBD4602B080BDC0468B
:1042C00080B588B000AF80239B02181C0121FBF74A
:1042D00015FF80235B01181C0121FBF72DFF3B1DFF
:1042E00020221A603B1D02221A713B1D03225A71C3
:1042F0003B1D00229A713B1D0122DA719023DA05E1
:104300003B1D101C191C00F03BFE3B1D40221A6097
:104310009023DA053B1D101C191C00F031FE3B1DDB
:1043200080221A609023DA053B1D101C191C00F036
:1043300027FE3B1D10221A603B1D01221A713B1DF6
:1043400000229A713B1D0122DA713B1D01225A7134
:104350009023DA053B1D101C191C00F011FE902360
:10436000DB05181C0521002200F0F4FE9023DB057C
:10437000181C0621002200F0EDFE9023DB05181C1E
:104380000721002200F0E6FE214B181C00F02CFC57
:104390000C23FB1800221A800C23FB1882225200E7
:1043A0005A800C23FB18E022D2009A800C23FB18C1
:1043B0000022DA800C23FB1800221A810C23FB1840
:1043C000802292005A810C23FB1800229A810C2330
:1043D000FB180022DA810C23FB1807221A820C4AF0
:1043E0000C23FB18101C191C00F02AFC084A80231F
:1043F0005B01101C191C00F0C5FC054B181C0121A9
:1044000000F0A0FC0123181CBD4608B080BDC046CA
:104410000030014080B584B000AFF8607A600B23B3
:10442000FB180A1C1A700B23FB181B78002B21D1D8
:104430009023DB05181C1021002200F06FFE7B6822
:104440001B0CDBB2181C00F093FB7A68FF231B02E5
:1044500013401B0ADBB2181C00F08AFB7B68DBB23E
:10446000181C00F085FB002000F082FBFB68012295
:104470001A7324E09023DB05181C1021002200F0A1
:104480004DFE7B681B0CDBB23F221340DBB2802267
:1044900052421343DBB2181C00F06AFB7A68FF2318
:1044A0001B0213401B0ADBB2181C00F061FB7B6887
:1044B000DBB2181C00F05CFBFB6802221A73BD46DD
:1044C00004B080BD80B582B000AF7860081C111CBC
:1044D000FB1C021C1A703B1C0A1C1A807B681B897F
:1044E000C22292039A187968FB1C1B78081C191CBD
:1044F000FFF790FFBD4602B080BDC04680B582B0D8
:1045000000AF78600A1CFB1C1A70FB1C1B78181C7F
:1045100000F02EFB031C181CBD4602B080BDC04637
:1045200080B584B000AF78600A1CBB1C1A800E23D3
:10453000FB1800221A807B681B7B022B12D1BB1C4C
:104540001B88DBB27A68101C191CFFF7D7FFBB1C55
:104550001B881B0A9BB2DBB27A68101C191CFFF780
:10456000CDFF19E07B68181C0021FFF7C7FF031C73
:104570001A1C0E23FB181A807B68181C0021FFF7F9
:10458000BDFF031C1B029AB20E23FB181B881343AA
:104590009AB20E23FB181A800E23FB181B88181CD6
:1045A000BD4604B080BDC04680B584B000AF786021
:1045B00039600023FB607B681B7B022B0FD13B68BB
:1045C0009BB27A68101C191CFFF7AAFF3B681B0CF2
:1045D0009BB27A68101C191CFFF7A2FF10E07B68E1
:1045E000181C0021FFF79CFF031CFB607B68181C54
:1045F0000021FFF795FF031C1B04FA681343FB60BF
:10460000FB68181CBD4604B080BDC04680B582B0B2
:1046100000AF78609023DB05181C1021012200F008
:104620007DFD7B6800221A73BD4602B080BDC04686
:1046300090B585B000AF786039607A683B68101C2F
:1046400000211A1CFFF7E6FE0F23FC187B68181CDC
:104650000021FFF753FF031C23707B68181CFFF732
:10466000D5FF0F23FB181B78181CBD4605B090BD65
:1046700090B585B000AF786039607A683B68101CEF
:1046800000211A1CFFF7C6FE0E23FC187B68181CBD
:104690000021FFF745FF031C23807B68181CFFF7F0
:1046A000B5FF0E23FB181B88181CBD4605B090BD36
:1046B00080B584B000AF786039607A683B68101CC0
:1046C00000211A1CFFF7A6FE7B68181C0021FFF7CB
:1046D0006BFF031CFB607B68181CFFF797FFFB68F0
:1046E000181CBD4604B080BD80B584B000AFF86032
:1046F000B960FB1D1A70FA68BB68101C01211A1CF6
:10470000FFF788FEFA68FB1D1B78101C191CFFF7C9
:10471000F5FEFB68181CFFF779FFBD4604B080BDAD
:1047200080B584B000AFF860B960BB1D1A80FA682C
:10473000BB68101C01211A1CFFF76CFEFA68BB1D38
:104740001B88101C191CFFF7EBFEFB68181CFFF7F9
:104750005DFFBD4604B080BD80B584B000AFF86099
:10476000B9607A60FA68BB68101C01211A1CFFF757
:1047700051FEFA687B68101C191CFFF715FFFB68D7
:10478000181CFFF743FFBD4604B080BD80B582B062
:1047900000AF021CFB1D1A709023DB05181C1021B2
:1047A000002200F0BBFCFB1D1B78181C00F0E0F998
:1047B000002000F0DDF9002000F0DAF99023DB059D
:1047C000181C1021012200F0A9FCBD4602B080BDDA
:1047D00080B582B000AF78600A1CBB1C1A807B6871
:1047E0001A89BB1C1B88D3189BB21B051B0D9AB2E0
:1047F0007B681A817B681B8903339BB2074A13408D
:104800009AB27B681A817B681B897A680449101CFC
:104810001A1CFFF785FFBD4602B080BDFC0F0000EB
:10482000FC20300090B585B000AF78607B681C89B3
:104830007B680E4A181C111CFFF71AFF031CE31AB1
:104840009AB20E23FB181205120D1A800C23FB18C6
:104850000E22BA18128806498A1A1A800C23FB18ED
:104860001B88181CBD4605B090BDC046F82030001E
:10487000FC0F000080B586B000AFF860B960BB1DCA
:104880001A8000237B6100233B61BB1D1B887B6179
:10489000FB68181CFFF7C6FF031C1A1E7B699A42AF
:1048A00005D2FB68181CFFF7BDFF031C7B617B6909
:1048B0009BB2FA68101C191C00F03CF87B699BB293
:1048C000FA68101C01211A1CFFF7FCFD00233B6154
:1048D0000CE0BB681B78FA68101C191CFFF70EFE71
:1048E000BB680133BB603B6901333B617B695A1E86
:1048F0007A61002BEDD13B697B61FB68181CFFF7E7
:1049000085FE7B699BB2FA68101C191CFFF760FFDB
:10491000FB68181C00F028F87B699AB2BB1DB91D12
:1049200009888A1A1A80BB1D1B88002BADD1BD4691
:1049300006B080BD90B585B000AF78600A1CBB1C86
:104940001A800E23FC187B68181CFFF76BFF031CF2
:1049500023800E23FA18BB1C12881B889A42F0D3BE
:10496000BD4605B090BDC04690B583B000AF78603D
:10497000C0467B680E4A181C111CFFF779FE031C09
:104980001C1C7B680B4A181C111CFFF771FE031CD2
:104990009C42EED17B68074A181C111CFFF768FE89
:1049A000031C1A1C7B681A81BD4603B090BDC0462B
:1049B000F8203000FC20300080B582B000AF786075
:1049C00039607B68181C0421FFF7B4FF7B681B89E2
:1049D000C22292039A1879683B68081C111C1A1CA1
:1049E000FFF7BAFE7B68181C0421FFF7F1FEBD46F5
:1049F00002B080BD80B582B000AF021CFB1D1A70F2
:104A0000FB1D1B78002B14D09023DB05181C042100
:104A1000002200F083FB142000F09CF89023DB05BB
:104A2000181C0421012200F079FB142000F092F8F8
:104A300013E09023DB05181C0421012200F06EFB1B
:104A4000142000F087F89023DB05181C04210022B5
:104A500000F064FB142000F07DF8BD4602B080BD7C
:104A600080B58EB000AF786039603B683B632B2324
:104A7000FB1800221A707B68181C01F0CBF9031C8C
:104A80007B627B6A7A68D3187B633B68002B0BD10F
:104A90007B6B5A1C7A6330221A707B6B5A1C7A63C8
:104AA00000221A70002351E03B6B002B07DA7B6B6E
:104AB0005A1C7A632D221A703B6B5B423B6323E0E6
:104AC0003B6B3B623B6B181C0A2101F073F8031C23
:104AD0003B633B6B0A22524253433A6AD3183B6210
:104AE0003B6ADAB21F23FB1830321A702B23FB18F3
:104AF0001B782B22BA18591C1170191C0C23FB1897
:104B00001F22BA1812785A543B6B002BD8DC0023B2
:104B1000FB620FE07B6B5A1C7A632B22BA18117868
:104B2000FA6A8A1A013A0C2179188A5C1A70FB6AAF
:104B30000133FB622B23FB181A78FB6A9A42E9DCEB
:104B40007B6B5A1C7A6300221A700023181CBD4626
:104B50000EB080BD80B582B000AF021CBB1D1A80B4
:104B6000BB1D1B88181C00F02BF8BD4602B080BD91
:104B700080B582B000AF021CFB1D1A70C0460F4BFF
:104B8000181C022100F044F9031EF8D00B4AFB1D4B
:104B90001B78101C191C00F013F9C046074B181C99
:104BA000012100F035F9031EF8D0044B181C00F069
:104BB0001DF9031C181CBD4602B080BD0030014029
:104BC00080B584B000AF78600023FB607B68C822AA
:104BD0005343FB6002E0FB68013BFB60FB68002B7A
:104BE000F9D1BD4604B080BD80B582B000AF786019
:104BF0007B68114A93420CD180235B01181C012170
:104C0000FBF7B8FA80235B01181C0021FBF7B2FA0E
:104C10000FE07B68094A93420BD18023DB01181C0B
:104C20000121FBF7C5FA8023DB01181C0021FBF7EB
:104C3000BFFABD4602B080BD0030014000380040E0
:104C400080B584B000AF786039600E23FB18002275
:104C50001A800E23FB187A6812881A800E23FB181C
:104C60000E22BA181188C12292010A401A803B68AC
:104C70001A883B68DB8913439AB23B68DB8813438D
:104C80009AB23B681B8913439AB23B685B89134312
:104C90009AB23B689B89134399B20E23FB180E22EC
:104CA000BA1812880A431A807B680E22BA18128832
:104CB0001A800E23FB187A6892881A800E23FB183C
:104CC0000E22BA1812881D490A401A803B6899883A
:104CD0000E23FB180E22BA1812880A431A807B682A
:104CE0000E22BA1812889A803B681A8A7B681A8248
:104CF0000E23FB187A6812881A800E23FB180E22E6
:104D0000BA18128804218A431A803B6859880E23F6
:104D1000FB180E22BA1812880A431A807B680E22EA
:104D2000BA1812881A807B689B8B9BB2044A134086
:104D30009AB27B689A83BD4604B080BDFFF0FFFF46
:104D4000FFF7FFFF80B582B000AF78600A1CFB1C44
:104D50001A70FB1C1B78002B08D07B681B889BB249
:104D6000402213439AB27B681A8007E07B681B8855
:104D70009BB2402293439AB27B681A80BD4602B030
:104D800080BDC04680B582B000AF78600A1CBB1CF5
:104D90001A807B689B889BB2084A13409AB27B6852
:104DA0009A807B689B889AB2BB1C1B8813439AB27B
:104DB0007B689A80BD4602B080BDC046FFEFFFFF12
:104DC00080B584B000AF78600A1CFB1C1A70002309
:104DD000FB607B68FB60FB680C33FB60FB68FA1CC4
:104DE00012781A70BD4604B080BDC04680B584B04C
:104DF00000AF78600023FB607B68FB60FB680C33CE
:104E0000FB60FB681B78DBB2181CBD4604B080BD9C
:104E100080B584B000AF78600A1CBB1C1A800F23D9
:104E2000FB1800221A707B681B899BB2BA1C12887F
:104E300013409BB2002B04D00F23FB1801221A70E1
:104E400003E00F23FB1800221A700F23FB181B78B6
:104E5000181CBD4604B080BD80B586B000AF786038
:104E600039600023FB601723FB1800221A7000230F
:104E70003B613A68FC239B01134005D07B681B68AB
:104E8000802213403B610EE03B68C022134005D0F6
:104E90007B681B68402213403B6104E07B681B6811
:104EA0003A6813403B617B689B69FB60FB683A682A
:104EB0001340FB60FB68002B07D03B69002B04D03C
:104EC0001723FB1801221A7003E01723FB18002296
:104ED0001A701723FB181B78181CBD4606B080BD3E
:104EE00080B582B000AF786039607B683A68DA617B
:104EF000BD4602B080BDC04680B500AF1A4B1A4A0D
:104F0000126801210A431A60174B174A5268174961
:104F10000A405A60144B144A126815490A401A6034
:104F2000114B114A126813490A401A600E4B0E4A7F
:104F3000526811490A405A600B4B0B4AD26A0F2142
:104F40008A43DA62084B084A126B0C490A401A631A
:104F5000054B054A526B01218A435A63024B0022DA
:104F60009A60BD4680BDC046001002400CB8FF08E4
:104F7000FFFFF6FEFFFFFBFFFFFFC0FFACFEFFFFE2
:104F800080B586B000AF7860396000237B61002374
:104F90003B610023FB6000237B617CE07B69012295
:104FA0009A40131C3B613B681B683A691340FB60E5
:104FB000FA683B699A426BD13B681B79012B03D09D
:104FC0003B681B79022B34D17B689B687A6952005D
:104FD000111C03228A40D2431A407B689A607B6886
:104FE0009A683B685B79191C7B695B0099400B1CD4
:104FF0001A437B689A607B689B889BB27A6992B2FD
:10500000111C01228A4092B2D24392B213409AB24A
:105010007B689A807B689B889AB23B689B79191C55
:105020007B699BB299400B1C9BB213439AB27B687D
:105030009A807B681B687A695200111C03228A409F
:10504000D2431A407B681A607B681A683B681B79F8
:10505000191C7B695B0099400B1C1A437B681A6022
:105060007B68DB687A6992B25200032191400A1C86
:10507000D2431A407B68DA607B68DA683B68DB7988
:10508000191C7B695B0099400B1C1A437B68DA6032
:105090007B6901337B617B690F2B00D87EE7BD46BE
:1050A00006B080BD80B582B000AF78607B68084AEA
:1050B0001A607B6800221A717B6801225A717B6832
:1050C00000229A717B680022DA71BD4602B080BD71
:1050D000FFFF000080B584B000AF78600A1CBB1CE5
:1050E0001A800F23FB1800221A707B681B8A9BB260
:1050F000BA1C128813409BB2002B04D00F23FB185C
:1051000001221A7003E00F23FB1800221A700F23EC
:10511000FB181B78181CBD4604B080BD80B582B05A
:1051200000AF7860081C111CBB1C021C1A807B1C81
:105130000A1C1A707B1C1B78002B04D0BB1C1A881D
:105140007B689A6103E07B68BA1C12881A85BD46A9
:1051500002B080BD80B584B000AF7860081C111C1F
:10516000BB1C021C1A807B1C0A1C1A700023FB60EB
:105170000023BB607B1C1B78BA1C128807210A40E5
:1051800092009340FB60BB1C1B88DB089BB2181C81
:10519000BB1C1B88DB089BB21A1C7B680832920080
:1051A000D358BA1C128807210A409200111C0F2202
:1051B0008A40D2431A40111C7B68021C08329200BC
:1051C000D150BB1C1B88DB089BB21A1C7B680832C1
:1051D0009200D258FB681343BB60BB1C1B88DB08E2
:1051E0009BB21A1C7B6808329200B968D150BD4648
:1051F00004B080BD80B582B000AF786039607A6855
:105200003B68101C191CFFF7D7FBBD4602B080BDE0
:1052100080B584B000AF786039600E23FB1800229F
:105220001A803B68181C00F0F5FD031C9AB20E238F
:10523000FB1801321A8079683A680E23FB181B8824
:10524000081C111C1A1CFFF715FBBD4604B080BDDD
:1052500080B582B000AF78600A1CBB1C1A80BD46C6
:1052600002B080BD80B582B000AF78600A1CBB1C64
:105270001A80BD4602B080BD80B584B000AFF86032
:10528000B9607A603B60FB69181C00F0C3FD031C29
:105290009BB20D339BB2FA68101C191CFFF7D8FFA4
:1052A000FA68F4235B42101C191CFFF7A3FF7B680C
:1052B0001A04BB681B041B0C1343FA68101C191C4E
:1052C000FFF798FF1823FB181B881A043B681B0480
:1052D0001B0C1343FA68101C191CFFF78BFFFA68AC
:1052E000FB69101C191CFFF793FFFB69181C00F0E9
:1052F00091FD031C9BB20D339BB2FA68101C191C64
:10530000FFF7B0FFBD4604B080BDC04680B582B097
:1053100000AF78607B68181C0421FFF799FF7A685A
:10532000DA235B42101C191CFFF764FF7B68181C12
:105330000421FFF797FFBD4602B080BD80B584B061
:1053400000AFF860B9607A601A1CBB1C1A80FB6859
:10535000181C0C21FFF77CFFFA68EA235B42101C43
:10536000191CFFF747FF7B681A04BB681B041B0C62
:105370001343FA68101C191CFFF73CFF1823FB1895
:105380001B881A04BB1C1B881343FA68101C191CC9
:10539000FFF730FFFB68181C0C21FFF763FFBD46C9
:1053A00004B080BD80B582B000AF78607B68181C07
:1053B0000421FFF74DFF7A68FF235B42101C191C84
:1053C000FFF718FF7B68181C0421FFF74BFFBD4651
:1053D00002B080BD80B582B000AF78607B68181CD9
:1053E0000421FFF735FF7A68E9235B42101C191C82
:1053F000FFF700FF7B68181C0421FFF733FFBD4651
:1054000002B080BD80B582B000AF786039607B6843
:10541000181C0821FFF71CFF7A68F6235B42101C5A
:10542000191CFFF7E7FE7A683B68101C191CFFF790
:10543000E1FE7B68181C0821FFF714FFBD4602B08F
:1054400080BDC04680B584B000AFF860B9607A60B6
:105450003B607B6A181C00F0DDFC031C9BB211331F
:105460009BB2FA68101C191CFFF7F2FEFA68F323CE
:105470005B42101C191CFFF7BDFE7B681A04BB6859
:105480001B041B0C1343FA68101C191CFFF7B2FE17
:10549000BB691A043B681B041B0C1343FA68101CFD
:1054A000191CFFF7A7FE2023FB181B881A04FB69B1
:1054B0001B041B0C1343FA68101C191CFFF79AFEFF
:1054C000FA687B6A101C191CFFF7A2FE7B6A181C85
:1054D00000F0A0FC031C9BB211339BB2FA68101CB5
:1054E000191CFFF7BFFEBD4604B080BD80B584B077
:1054F00000AFF860B9607A601A1CBB1C1A80FB68A8
:10550000181C1421FFF7A4FEFA68D0235B42101C7C
:10551000191CFFF76FFE7B681A04BB681B041B0C89
:105520001343FA68101C191CFFF764FE1823FB18BC
:105530001B881A04BB1C1B881343FA68101C191C17
:10554000FFF758FEFA68FB69101C191CFFF752FEA2
:105550002023FB181B88FA68101C191CFFF74AFE51
:10556000FB68181C1421FFF77DFEBD4604B080BD0A
:1055700080B584B000AFF860B9607A601A1CBB1CBB
:105580001A80FB68181C1421FFF762FEFA68CB230F
:105590005B42101C191CFFF72DFE7B681A04BB68C8
:1055A0001B041B0C1343FA68101C191CFFF722FE86
:1055B0001823FB181B881A04BB1C1B881343FA68AA
:1055C000101C191CFFF716FEFA68FB69101C191C49
:1055D000FFF710FE2423FB181B881A042023FB1856
:1055E0001B881343FA68101C191CFFF703FEFB68A5
:1055F000181C1421FFF736FEBD4604B080BDC0461E
:1056000080B582B000AF786039607B68181C0821D3
:10561000FFF71EFE7A68CC235B42101C191CFFF7B3
:10562000E9FD7A683B68101C191CFFF7E3FD7B68F5
:10563000181C0821FFF716FEBD4602B080BDC0460B
:1056400080B582B000AF786039607B68181C082193
:10565000FFF7FEFD7A68EB235B42101C191CFFF775
:10566000C9FD7A683B68101C191CFFF7C3FD7B68F5
:10567000181C0821FFF7F6FD7B68181CFFF774F96A
:10568000BD4602B080BDC04680B584B000AFF860B2
:10569000B9607A60FB68181C0C21FFF7D9FDFA6825
:1056A000E4235B42101C191CFFF7A4FDFA68BB68D9
:1056B000101C191CFFF79EFDFA687B68101C191C52
:1056C000FFF798FDFB68181C0C21FFF7CBFDBD46CA
:1056D00004B080BD80B582B000AF786039607B686F
:1056E000181C0821FFF7B4FD7A68DD235B42101C0B
:1056F000191CFFF77FFD7A683B68101C191CFFF727
:1057000079FD7B68181C0821FFF7ACFDBD4602B08F
:1057100080BDC04680B584B000AFF860B9607A60E3
:105720003B607B6A181C00F075FB031C9BB21133B5
:105730009BB2FA68101C191CFFF78AFDFA68F22365
:105740005B42101C191CFFF755FD7B681A04BB68EF
:105750001B041B0C1343FA68101C191CFFF74AFDAD
:10576000BB691A043B681B041B0C1343FA68101C2A
:10577000191CFFF73FFD2023FB181B881A04FB6947
:105780001B041B0C1343FA68101C191CFFF732FD95
:10579000FA687B6A101C191CFFF73AFD7B6A181C1B
:1057A00000F038FB031C9BB211339BB2FA68101C4B
:1057B000191CFFF757FDBD4604B080BD80B582B00F
:1057C00000AF78607B68181C0421FFF741FD7B68FF
:1057D000064A181C111CFFF70DFD7B68181C0421DC
:1057E000FFF740FDBD4602B080BDC04600FFFFFF91
:1057F00080B584B000AF78600023FB60334BFB6062
:105800007B689B79002B4FD0304A304B19687B68FE
:105810001B68DB430B4013602C4A2C4B59687B6898
:105820001B68DB430B4053607B681B791A1CFB68C9
:105830009B18FB60FB68FA6811687A6812680A4373
:105840001A60224A214B99687B681B68DB430B4036
:1058500093601E4A1D4BD9687B681B68DB430B4075
:10586000D3607B685B79102B0ED1184A174B99686F
:105870007B681B680B439360144A144BD9687B68A0
:105880001B680B43D3601DE0104BFB607B685B79AA
:105890001A1CFB689B18FB60FB68FA6811687A6841
:1058A00012680A431A600DE07B681B791A1CFB68BA
:1058B0009B18FB60FB68FA6811687A681268D2432B
:1058C0000A401A60BD4604B080BDC04600040140D5
:1058D00080B584B000AF78600F23FB1800221A70E7
:1058E0000A4B5B697A68134004D00F23FB1801222E
:1058F0001A7003E00F23FB1800221A700F23FB1805
:105900001B78181CBD4604B080BDC0460004014091
:1059100080B582B000AF7860024B7A685A61BD46AC
:1059200002B080BD00040140B0B584B000AF021CDD
:10593000FB1D1A70BB1D0A1C1A700023FB60BB1DE7
:105940001B78032213409B000F229A40131CFB601C
:105950001849BB1D1B789B08DBB2181C154ABB1DE0
:105960001B789B08DBB202339B009B58FA68D2433A
:105970001A40831C9B005A500E48BB1D1B789B0885
:10598000DBB21D1C0B4ABB1D1B789B08DBB202332C
:105990009B009A58FB1D1978BB1D1B7803242340DC
:1059A0009B0099400B1C1A43AB1C9B001A50BD4630
:1059B00004B0B0BD0000014080B584B000AF786095
:1059C0000023FB607B689B78002B39D0234A7B68DF
:1059D0001B789B08DBB2C0339B009B58FB607B6845
:1059E0001B781A1C03231340DB00FF229A40131C70
:1059F000DA43FB681340FB607B685B789B01FF2206
:105A00001A407B681B78191C03230B40DB009A406B
:105A1000131CFA681343FB6010497B681B789B08D2
:105A2000DBB2C0339B00FA685A500C4B7A6812788C
:105A3000111C1F220A40012191400A1C1A600AE031
:105A400006497B681B781A1C1F23134001229A40C9
:105A5000131C80228B50BD4604B080BD00E100E0E5
:105A600080B582B000AF78607B68042B06D1084B0C
:105A7000074A126804210A431A6005E0044B044AED
:105A8000126804218A431A60BD4602B080BDC04638
:105A900010E000E0002243088B4274D303098B42DC
:105AA0005FD3030A8B4244D3030B8B4228D3030CEE
:105AB0008B420DD3FF22090212BA030C8B4202D390
:105AC0001212090265D0030B8B4219D300E0090AB8
:105AD000C30B8B4201D3CB03C01A5241830B8B42C1
:105AE00001D38B03C01A5241430B8B4201D34B03AA
:105AF000C01A5241030B8B4201D30B03C01A52410F
:105B0000C30A8B4201D3CB02C01A5241830A8B4293
:105B100001D38B02C01A5241430A8B4201D34B027C
:105B2000C01A5241030A8B4201D30B02C01A5241E0
:105B3000CDD2C3098B4201D3CB01C01A5241830994
:105B40008B4201D38B01C01A524143098B4201D3CE
:105B50004B01C01A524103098B4201D30B01C01AF9
:105B60005241C3088B4201D3CB00C01A5241830873
:105B70008B4201D38B00C01A524143088B4201D3A0
:105B80004B00C01A5241411A00D201465241104600
:105B90007047FFE701B5002000F0FCF802BDC046E9
:105BA0000029F7D003B5FFF775FF0EBC4243891AF1
:105BB0001847C04603460B437FD4002243088B425C
:105BC00074D303098B425FD3030A8B4244D3030B84
:105BD0008B4228D3030C8B420DD3FF22090212BA49
:105BE000030C8B4202D31212090265D0030B8B42C5
:105BF00019D300E0090AC30B8B4201D3CB03C01AAF
:105C00005241830B8B4201D38B03C01A5241430B89
:105C10008B4201D34B03C01A5241030B8B4201D379
:105C20000B03C01A5241C30A8B4201D3CB02C01AE4
:105C30005241830A8B4201D38B02C01A5241430A5C
:105C40008B4201D34B02C01A5241030A8B4201D34B
:105C50000B02C01A5241CDD2C3098B4201D3CB01F2
:105C6000C01A524183098B4201D38B01C01A5241A1
:105C700043098B4201D34B01C01A524103098B42A5
:105C800001D30B01C01A5241C3088B4201D3CB0090
:105C9000C01A524183088B4201D38B00C01A524173
:105CA00043088B4201D34B00C01A5241411A00D223
:105CB00001465241104670475DE0CA0F00D049428C
:105CC000031000D34042534000229C4603098B42FC
:105CD0002DD3030A8B4212D3FC22890112BA030A84
:105CE0008B420CD3890192118B4208D38901921106
:105CF0008B4204D389013AD0921100E08909C3098B
:105D00008B4201D3CB01C01A524183098B4201D38C
:105D10008B01C01A524143098B4201D34B01C01A77
:105D2000524103098B4201D30B01C01A5241C308EF
:105D30008B4201D3CB00C01A524183088B4201D35E
:105D40008B00C01A5241D9D243088B4201D34B0079
:105D5000C01A5241411A00D20146634652415B10BB
:105D6000104601D34042002B00D54942704763469C
:105D70005B1000D3404201B5002000F00BF802BDDB
:105D80000029F8D003B5FFF715FF0EBC4243891A6E
:105D90001847C0467047C04670B50F2A32D9041C58
:105DA0000C430B1CA40731D1151C041C103D2D09FC
:105DB00001352D0149191E6826605E6866609E687F
:105DC000A660DE681033E66010349942F3D10F23E9
:105DD00045191340032B1BD91C1F0023A4080134B1
:105DE000A400CE58EE500433A342FAD1ED18C918DE
:105DF00003231A4005D00023CC5CEC5401339342BA
:105E0000FAD170BD051C002AF5D1FAE7051CF2E7AE
:105E10001A1CF8E710B5830727D00378002B26D08B
:105E2000031C032102E01A78002A1CD001330B4224
:105E3000F9D119680F4A104C8A188A4322420FD1AF
:105E4000043319680B4A8A188A43224208D1043362
:105E50001968084A8A188A432242F1D000E00133C7
:105E60001A78002AFBD1181A10BD031CE1E70020A4
:105E7000FAE7C046FFFEFEFE80808080F40100004D
:105E8000BC02000000000000000000000000000054
:105E9000DC050000D0070000E8030000F40100006A
:105EA000BC020000B80B000000000000B80B0000AE
:105EB000DC050000D0070000E8030000F40100004A
:105EC000BC020000B80B0000A00F0000B80B0000DF
:105ED000DC050000D0070000E8030000F40100002A
:105EE000BC020000000000000000000000000000F4
:105EF000DC050000D0070000E8030000F40100000A
:105F0000BC020000B80B000000000000B80B00004D
:105F1000DC050000D0070000E8030000F4010000E9
:105F2000BC020000B80B0000A00F0000B80B00007E
:105F3000DC050000D0070000E803000071776572FF
:105F4000747975696F7000006173646667686A6B65
:105F50006C0000007A786376626E6D0020000000AD
:105F6000373839003435360031323300302E0000F6
:105F70004E6578742064656D6F20696E20000000A6
:105F800073000000534B49502D3E0000447261776E
:105F90002074657374000000434C454152000000BA
:105FA00000010304050608090A0B0D0E0F11121358
:105FB00014161718191B1C1D1E2021222425262704
:105FC000292A2B2C2E2F30313334353637393A3BB2
:105FD0003C3E3F40414344454647494A4B4C4D4F68
:105FE0005051525355565758595B5C5D5E5F606225
:105FF0006364656667686A6B6C6D6E6F70727374EC
:1060000075767778797A7C7D7E7F808182838485BE
:106010008687898A8B8C8D8E8F909192939495969A
:106020009798999A9B9C9D9E9FA0A1A2A3A4A5A688
:10603000A7A8A9AAABACADAEAFB0B1B1B2B3B4B57D
:10604000B6B7B8B9BABBBCBCBDBEBFC0C1C2C3C382
:10605000C4C5C6C7C8C9C9CACBCCCDCECECFD0D196
:10606000D2D3D3D4D5D6D7D7D8D9DADBDBDCDDDEB3
:10607000DEDFE0E1E1E2E3E4E4E5E6E7E7E8E9EAE0
:10608000EAEBECECEDEEEFEFF0F1F1F2F3F3F4F517
:10609000F5F6F7F8F8F9FAFAFBFBFCFDFDFEFFFF59
:1060A0005269766572646920372E3022206E6F2027
:1060B000746F7563682064656D6F00005269766562
:1060C00072646920372E3022205254502064656D4E
:1060D0006F0000005269766572646920372E3022A5
:1060E000204354502064656D6F000000526976654E
:1060F00072646920352E3022206E6F20746F7563B4
:10610000682064656D6F000052697665726469206D
:10611000352E3022205254502064656D6F000000EF
:106120005269766572646920352E302220435450BE
:106130002064656D6F000000506C656173652054CC
:106140006170206F6E2074686520646F74000000B9
:10615000506C65617365205461702066726F6D20AC
:106160003220746F203520706F696E7473000000E8
:10617000504F494E54530000446966666572656E1F
:1061800074207479706573206F66207370696E6E09
:1061900065727300506C6561736520576169742086
:1061A0002E2E2E004C270008D2240008A825000817
:1061B000F62500084426000892260008E02600087C
:1061C000C8290008762D0008042F0008B42F000805
:1061D000223400087C34000858380008FC3B0008D2
:1061E000203E0008D82B0008142A0008462A000880
:1061F000782A0008AA2A0008742B0008A62B000899
:10620000789CED9D3996EB2814861D2BF02A1C13E3
:10621000F8ADC2A9B50E4515681F4A14781F4EB4D3
:1062200014056CA2DF39CF0ECA6D0DC0052E70D1DA
:10623000E42A9BFFF4E9579600C1FDC43CE8F1480D
:10624000FA3835E5578EEB9C9FCFE7A326C69EFF15
:10625000F9B5778BB1BC7975723F4CB507C72A6227
:10626000FCD549FE24E55BE37D8AAF971CDE08ADD3
:10627000F78C17CB4EA127CD9BE7DE4EE7F5125FDB
:1062800067E3338EEB3DE3C51229CCE41561D7CC2F
:1062900006CC3687DB69BDC427BE9ADA7D665B7F94
:1062A0007565ED6A894F7C354973ECB3F5B577C7F1
:1062B000633125BE9A4A718B5D9AB57529BD7CEB19
:1062C00063BCF29A9BA124BE50B279B549CCB88F79
:1062D000AFA41FA52CE77A82125F28610EB64DD4B9
:1062E000CE8BF37DAAC61294F8F612E658B1C70217
:1062F000B50A5F0D70E2AB499823EF7F2893B1BEDA
:1063000085AB4CCED8224DDE75F842C0B568CB6D5A
:106310005422BD40085FD18275D6BF47F843128032
:10632000265F846FBE0E5F3820265A73EB75C15E00
:106330002D9BAF7BFC4AE4DF23FCB1173DD4D2BCDC
:106340003057ABF0CDC6E2E75364F3754BE70B6C07
:1063500026F3AFE8B62ED2655D2BFF667C89D8FDAB
:1063600012C5F0BDEC215F730402987C9921091AD3
:10637000DF09436AE512B1FB258AE1DB8C6EFBD6AF
:10638000C8FA7CBF487CF7A109667BA279A3F6FF17
:106390008F50145FD8FFF5F15DA67C167C2FC8BD29
:1063A00072C2A38ED2CF12B1FB25FAED7C231A4B19
:1063B0008D8CF112B1FB259ACED72C8E572B9FD7FF
:1063C000E3CBEBCBA031BEE2E7C51AA9764B8671D1
:1063D00031E3C99B8B4FBE4E99DF2BA73A7C2644F5
:1063E00022516670A671E3FC5BAECE578C6F64E3FE
:1063F000F806933363F42A3A57135EF0729B8727AB
:10640000D9F647D44EFC2BE055FA2A19791A8E3268
:10641000BE41CEBF8BF2D5878C8D7B33F98A0B239F
:10642000DF8B6A8D5353206741F478967B5ACB1EDD
:10643000798FC28B64C6B835418740F6F8A49D4475
:106440008D6F73562B27FB92A6362FCCD5C030CB41
:10645000B6E30B16A85047A4D58A34865E0D58DDE6
:106460005E5E46F0DA081344F40DA3F9AE2F513EF8
:10647000AFC8D79C5F504E8819B8550520F070A65C
:10648000DBDD044C793386E232AEE34F995F90A9AD
:10649000279B749636289FADF9A3A374437B89FF8D
:1064A0004803820C1F637A636E83B482B103D3D234
:1064B0001F313C473E425EF944BEA04EC39A75561A
:1064C00090BAD107F17D8C322D7D242FDDA358D4D5
:1064D00043125F2155B45232B01A3201D937769146
:1064E0003878106D58BD896C5B75A2AD9F1CD5FDC9
:1064F000E02D17A29B384AA3F5B7AC7F5D156A3033
:1065000044386346B538F22046F2D9C07788581728
:1065100044F3ED461F441F8BD38D1CA197F07534B7
:106520008871291C201A2A6B51AB6139DFC1693E81
:106530001AF80EADC95788D38D1C2161FD6DF98203
:10654000DA137B30D44539E5C8D5ACE43EA9F74031
:106550007682550CBF5A8F4F10C92CF739E40DFBCA
:10656000057CB1E9BCF5F8C2EA3310A0349E160BE5
:10657000D9040E75A1D57263CB6BE8C92AA373BF8A
:106580004399660A5F0E9FBE01DFFD4BF8AA0C8C93
:10659000D60C4A1755346A51CB8851B34657902BC5
:1065A0000EB556525CFAC97C5F937F6123D61B9E61
:1065B00072A6C530F125EAF222BE0A5CE65BE9016B
:1065C0008622F4A825BE34BD8C2F2D032B477A04D8
:1065D000135FA29A57F175A2D36280D7BE892F5953
:1065E000AFE35BBBD8014917662B2CF1258AC43772
:1065F000622EAB26F31D7B3EDDDD2F476060B78644
:106600007927F1A589C4779FFB17A82821449C7C92
:10661000C7318ACC9936300A62CE43FC5EBE0F1871
:1066200068532A851E324D34BE1324F3A47B7F1990
:10663000DB8B913F9C923BFBBE0BDFF5B51A5F995C
:1066400030375F30D1CF91C77324301935E195D5FC
:106650007EC981B20FE78B5581B3F8CA503CFB432A
:10666000E5CC5F866543358669FB8C5C58B14F7C11
:10667000917B73F8AA0AD3C317CC02D976687D3709
:10668000135FA256E20B962CFAF677E79807EB1EFB
:1066900092B9135FA2DAC5F96686E97C7CC5D3336B
:1066A000BB8A95D64567BE135FA296E76B5ACE7B31
:1066B0003E83CCA49979F72867D5B1BA39F125AAD8
:1066C000F51931D68643928CB0BC7CB9F0635A027E
:1066D000AC7DE258D4125F9A38856F685F0674B358
:1066E0002F8D75F7FEF355BE6436D5CDAD16D5A109
:1066F000835B892F5124BE39478F4783EB0B99F376
:106700008C0D3F5F30D10F4DD1A88A198D76E24BA9
:10671000148DAFC333DC1EE51A430E9D8FA4484190
:106720007B33192E3E6E277D05F77E0925BE96C266
:10673000F347707CDCB5CE2674FE1516826B5A5F6B
:10674000458D3A3E89C427F11D45981F54D5A4F3C1
:10675000BCA6105F6CA29F498B39DE9A37E0CB63F1
:10676000233E49A2FE9BC8575B67CE5117C1F3EB8E
:10677000A47F0933987D135FAAE6F2855BB0708031
:1067800041BEF644BF0AD255E827BE44CDE50BD73B
:106790009FE3EEC2E74F3203A7675E5046EDF7F284
:1067A00015A9E5AED0BE07851E4AD4F834ECAC047A
:1067B000DAFA1CD855C1B25B982FE867C128ED3DC5
:1067C000DB0BDF91EFFD76BBFDA7EBEFED769F09CD
:1067D0007A365F6D2B1FF6BD90205F9081BBDE1077
:1067E000DE6332A2F6DBF91AA3EA7793ACA6DB9D4F
:1067F00096344C1EE353D7D7293C9829087CD506FC
:106800008FFD03D8C6B3BDFFB7F365E0609D6F2F62
:10681000DBB98C17E00BF75ADB46A39CFFAC3604C0
:1068200097A04FEDF1F08BF9765D4A70F54E813B04
:1068300003F1027CB58DD0965B0A5FB8451FFCE979
:10684000F6F0A3F8F248BE20CEA4AC3B0BB127B1C2
:10685000F4F5CFF0D835B38D453ABF1DD98E8FAE44
:10686000D9B1028D1F0622F355FB07039BD091F38C
:10687000CD3C7CFFA891DC58BA03E2B806D7227C55
:106880007D6D2C125FB8E95AFCC93DEE1BE9969567
:1068900034C9D78ECC17EEB0F049552824BE322229
:1068A0001125B3A1984CBC0C5FAD8DC5F5F450F823
:1068B0002219D8FBD0B8E355B404D2F9324F70A8EE
:1068C000487C477D4FA6DB67E250DCCD98CCE5EBFA
:1068D0006E63D1F8DAC0B8F779D1B69FC0F7CB179D
:1068E0001EA608BE938AE629843D898DDA7FE46C72
:1068F0006311BF9F621A33B09E9F748615D404BE85
:106900006DE60B101199EFBCCC1B45D893D8B8FDA0
:1069100065D0E2100EF5FB3886AD428F6391B69FCD
:10692000C037FA10262ADFE9356F3C614F6223F742
:106930000F8AA3FEBBFF816451F9EAABBD82DB7114
:10694000620FA79AC2977A0A931091EFECB2398638
:10695000B027B1B1FB4319482A9757C947A168A688
:106960000A3F2DB2849EC4B79B1D8B28A4697C313D
:10697000BCB7DBFD3E4E297C7FDFEFD640B45BA188
:10698000B6B4C7A0B17CF13616D99E70B54FE8D425
:1069900024E19E6EFC497C234FA0A49C1FFBF86B56
:1069A000A275CD207CD32807B2301B2382DC8ADE7F
:1069B000DF8DB6B1E8DFA703BE498F6B8F11796B0E
:1069C0001ADFAED6A13F84927F0D38A1C10AFFC461
:1069D0000381F0927CB532535C9313C441BE6A2AA2
:1069E00099927D3B35F41690CD9778FA342F9927FC
:1069F000585DD293BC62F28D823B283CFFE00BC80D
:106A00008A5AD28A028573D44872A8C5EDCCC26D69
:106A1000E2BBA1544E8C9E2708E4E27F83ABA6AE76
:106A2000EBCBB012BDED0E55241FD697B4802422B7
:106A30009B6EDBD465397C77A12CEB0BDA6DF623EA
:106A40001EB270C3D492705873BCEFC7797F8EEEBC
:106A50001A09A9A63CEF0D1ADD3726595E37DC0A64
:106A6000C28778A8856BAC4148EA9024CDD23742E2
:106A7000B77936DE3A1C781BBD876C2E2BF7101EBB
:106A800083BE303B38BE4D1A3F5956D1DC122730F9
:106A900072A3B4F664E231F4C6ECD57DD4E77A5F34
:106AA000A39B91796B95CB423DEC6CFFC7F8105AD4
:106AB00090F0E30211D3BAFA493374D7F1C6EFADBF
:106AC00066B51D1EA6BFB233DC88F2E193BEE5FABF
:106AD0002A69657339E58BCA9951503B9BD360B8DD
:106AE0008337655E2EF2A1BB24AF6EB28BDA8FA026
:106AF0004DC0DB1336E6D59CC5F48C05D349137421
:106B0000576573D4A83922FDBB84CEB6167D054FD8
:106B1000D27C297BE34573CC24A4F9455427E19426
:106B200089B7D24DE0E5470D6537AAC1F2B2AEBBD9
:106B300011C5BA2E7326507B81674C277CFF9710B6
:106B4000BF54B25F6A64C4D21EA1E256DF15CBE91E
:106B500099D19A760F5DFE05F3CB89F63A12D948A2
:106B60005B72628E5A00B55F9402DBD85C199E2975
:106B70004E55F23A127B79BFD4363A0FDC414D1EA6
:106B8000249C3173FBAC7F1631E5DE75A58E2A2679
:106B90000DF673FFE8658F9F59AF893313A7CCBB00
:106BA000B2C41EC960D695E2DE41AE1E70667FC5D6
:106BB000FDFB66AEF04AEDAC0D349E3494F3285FD5
:106BC00084F547D8D401AC8B6F911BD292A6680094
:106BD00065E7B69028A321D33FDDC027FB4CD2D474
:106BE000B596B2C8BC3B8AB2907F22E134E9BF902F
:106BF0004A7B4C2242DE423A1B2AE209A8F8914F16
:106C00008D5192A67A1A0029F585610FE6D8D2A196
:106C10000E6D5B4F22AA757FC18B2AD23AEF7304A7
:106C2000B096A5351D4B09E9A6468BB49D2E63256C
:106C30002785D676EFCBEC38D114DFA4A47A890867
:106C4000B96DA3A34156BEC8A7C9F83188B7173399
:106C500056F2206AFAAEF836A5F36EB7ABE27C5C6A
:106C60009F5E480E0BAAC321CCB50063679E4F12EE
:106C700079C324F3ADD868CB61DDD746A5F3FBF328
:106C80005D4ECF3A932C864C4DF58BEE8490BB6BCA
:106C900028F18D5178D26150BFA43A5353CB4D5354
:106CA00097F971AF16D16FB6DEBD288A6B9C8F4FF6
:106CB000E61B7D6A41BF59659F59AFC50FDEAEF235
:106CC000D17C1F9CC51246C55F9D0EB73E9BEFCC85
:106CD000AF7E8EB25AF46D519C0615A7A2184CF1E6
:106CE000FC0B569DD7E78DE1AFA7DBD1B5E6E07988
:106CF000BF90C1885BCF0BCFF2B97A7A004EBB67E9
:106D00000CA576A5DC17A30FC85745EB24A3A54215
:106D1000793A84F7453D50413F2ACC939288DB096C
:106D20006A0CBF7AFE695A47F86861FA62EB1DB2D5
:106D3000A2CB684BD676866AA7AB4FCDE1693EC33E
:106D40004DF7EF153A84A6D899BA3E44FBAA153FF1
:106D5000D5D31EE323A00E22FCD1E1D5081046674F
:106D6000E06B7B7786A95F6D5D11BE1AA91A1F546F
:106D700005A3B39CF879DE0A5BABEB6B25BF2FCC88
:106D800070BE2D62D2415620BB876C3F5F45A0E2AA
:106D9000EF1EF6C1F4707A40BEAD797BA765198B02
:106DA0006F1FDD9379F18026F08046784CB65E96B1
:106DB000B7A3F340749654F4E96E50F627A52C3B24
:106DC000F796C2F9EA56F5E6DF8EEC6E2C0C7A6F78
:106DD000CADD50DCA106567C6D80F075426EEF7CFA
:106DE00061DA6CEC8B5D7AAD0C5C0CAE43D159541E
:106DF0002DB205942A7BB35997A256E930C41CE7FB
:106E00007BEA0A372923940A84329849B0ECDFA13F
:106E100093F6C7D0EA51BA0E76547C0FDAA35AB370
:106E20003D55E8DEAB1E651F081AA611B7A21FB4B8
:106E3000843A8008828489EC1B8ACEC29ADECCB266
:106E40001B923B7D10A208F0B5DA1F321458601D6A
:106E500074BE8F317F14EABDAF0C0B0D6E35BEF0E2
:106E600051D7A2D06A3CC3C06DFF7C7798AD7ED568
:106E7000AE3C4FA0B23E6997656D02A3633E69695F
:106E800011260D5121231B9BF01DDA58D54E991A5E
:106E90006161E65FC7A3443457E1DB1395AE65F645
:106EA000DD9AEFC42C8C8D3B6FC25735D2AFE08298
:106EB0001DC0EBF96A19B89011DE9CEF330B67B176
:106EC0005B11D19DDEDBF0150D14196817620164AA
:106ED000F23DE9F72BA4FF0B7E2ABE46984EBE5525
:106EE000A1E9202B0E5003B78A75771F383FADCF2D
:106EF0007742439A63A16CC47768A72BDF66AFDB48
:106F0000E46BDDB7FBBFE0A7E26BC8C9D7767A5068
:106F1000418DD10465B5DDCB589FEF83C79D618C52
:106F20004F1C6EC5B7D8693F437C6D8B5AFD5FF02F
:106F30007341BE8A2A20FD1ABE71FB891DF3C21B54
:106F4000F1BD1A90DC2C840B73B0C2EA97423B2C43
:106F5000C85762854DAD17F1952DE93066D7B4FF5E
:106F6000367C5BD32A7D8F55D7C39C5F00F7CC0A54
:106F7000CFC9170F13E55BE8E1CB018B912BCCBE9A
:106F80007D82ECA0375177E2D574BC1BF1EDDEFFBA
:106F9000BE5522FCE32D50E7FC91E99CD47E56615E
:106FA000A27CB5F911C07704ABF59402CDF9751543
:106FB000EE0D33EEF4BC09DF7160E3B093C1FE6007
:106FC000BE03592DFBBE962F72A69926EFD7C2B6E7
:106FD000E02B0636C0545288EF099FC002D15C8F67
:106FE0006F3FACA165DF57F37D7447A6A1F57086AE
:106FF0006D2485EAD252498911C42EA7A9ABD58147
:10700000C0D70805D8506155B3839DD58B4A93A846
:10701000F39E7F8EFD5F2B0252857E7B808187E908
:10702000E40B225C1D205FD1B403693DD84153C1FC
:107030002CA6763CCFD2289A03ABADAC39B59E894D
:1070400073FECDCDD7D055F105C5B21A81B67D54AA
:10705000EA6A8BB485ADF6B3215798385F3BD98087
:107060006F2B62218534CDC3409617D74E267CFE08
:10707000F9156CE659936AE84CF9909C08BEE31C3C
:107080006B35F8D21AA2036B9B5097C32B69592B0F
:10709000025A4ABCBE819C7CEDB9C48319BC36A29D
:1070A00062779042865D4B6D9DB34E79195EEDDE41
:1070B000BBD7A37E68DD57E97C4FE3C50A96C97D3F
:1070C000B882858DA8CFEB9564A9E7B083FEA2E2D4
:1070D0009ED1CB8EF1E7D624A64DE8EE0C4F488624
:1070E000A7D8F66708EFD62157DDDDBE9D3EC72A3B
:1070F0009DDBBEC02FBC4329FFF4F6365D9D51E4F5
:10710000BAE15B4B8DEB11C8237DCEDF5E3B63FCA8
:1071100030E9BD94F8BEB712DFF756E2FBDE4A7CD9
:10712000DF5B89EF7B2BF14D7A3FFD0FBB9DCAB42E
:10713000789CED5A3B72EBB812CD19702908B41047
:1071400006F03E1C5055C3554C600666C05D28A035
:1071500003ECC38111209D17BCE0C50A38E80F80FD
:1071600006254BB4E77ADE55559FE0162F0C348088
:1071700083FE025A578542A15028140A8542A15025
:1071800028140A8542A15028140A8542A1502814C7
:107190000A8542A15028140A8542A15028140A8564
:1071A00042A15028140A85E27110266BDAB63576B2
:1071B000F0BBFABB3962FACE4CD38C98C43C6EE675
:1071C000B6EFC87B2404DB1618B763041C4ADB84C3
:1071D000AF4FE51A9AA5E94B5B9AB9D971C6FBD4B2
:1071E0002061B27BCE6E0E5F12BA13E162EAA9692A
:1071F000259AE1BE10EAF9B54D2386348BCD4D2E8C
:10720000CF7C575E104A10827721841BBD5DDB88DE
:10721000693E951927BEDB691F9C35790BF642AA9A
:107220006DB7E8D73B08A4F9EF5F5F4A9ECCE6153F
:10723000996C49EF77888E0AC13D665488B6891AE1
:1072400032DFE8ED9ABBC6895BD9BBFA5B70B0B59B
:10725000869578889BDAA8AB692F71CFDA4805BB91
:10726000E5EBAB29EE29711AB235993BF20EA0F28B
:107270005E2EDA98CF793EB68D3B9A5D0B3ADCF8FC
:10728000BBDBE346633783DB48DCD2FA24D397DAEF
:10729000BCC382C9FAFBAFEB73283C7F70535FCC51
:1072A000E8A63C4747812B0BDDE0425CFA0DAF308E
:1072B000B5ADDBA1CE71FBF38D5E91BEFB9E07C425
:1072C00034CDF1D8DAC0FF8D7B02A645009BD226D3
:1072D000BB7E8CE89255DF5D5DC4F875FF5C7C7108
:1072E000E6B91CEE4D79BE113CA7919F33E49BF8A3
:1072F000B7E6B8633DD1A9DE9A7457B03F820B2838
:107300004E209AA889B124CACE2D89E597715C00D8
:10731000E32E8526B358BECEF354787EDFB6DCE686
:1073200099FA59A1F2B0F6F0F90AA7D5ECF11A369C
:107330005C3FAC23587DB04F9FCE20E0805701DBEF
:107340003633C490464645A439B2EC1189E8D73BA0
:10735000CBFB26CF381F9D1233664ACB4D79B4D272
:107360005EA6DD6D0E60F396AA3E6E7C07CD319C65
:10737000AEE69AD2CF576DC54DE1AA1870A3A27799
:1073800020CFEC4A9CF389E6C5A70D78DA903997AF
:107390006150473839030D3377797671A4AB3A21C0
:1073A000A19DE09923EA461E4DB95E8CAC8EC2A623
:1073B0004033C5BC233B3A779CD0DEBD70077E903E
:1073C000AB87B43A0B9D86DC6DCEEE753D365768C3
:1073D0008650D7AC69D53255C0505EA618F83FA587
:1073E00013733ACAE52FB5E3984D32F422996D78BC
:1073F000593B03106420A8A3CF1156280CFEFF5957
:10740000F04C0A8E3CE7F4A5E4D86911D6E4559413
:107410006558E6C2340793F2A9C8057C46A95D0900
:1074200031C73A8D06BE0CE53B9189E47FC3015B11
:10743000516274B726AC1BC434F1C0EE210AAC23F0
:1074400018565FF96098DF50120E5A7B5F29E6D913
:107450009AEEB94FBE32ED0FB79DBA508AD07FF089
:1074600039E5D133F543531864F193164DE1805C4F
:10747000D3521A9E71965E6A3821D1279ACA760C29
:10748000EDDA3647C7D52558BB75D4DFAE9E064327
:107490003C828D3BAE0D8193262EBCA130E7045378
:1074A000965284296FD516B5758D7106D90F98C27D
:1074B000D5A9AF138B8DA7E486A7235C64747C44A5
:1074C000A422A73A6FF5CB29C6C42A4F65A4FA8532
:1074D0005AE3510C85B1D2DE43B971AC06263F4A5E
:1074E0001C9E6814CC3008E2E9685D559C120D4181
:1074F0003665A568DBA7156DB6A70A160A05D2473B
:10750000079AE41A54D5B98155ADDE30A747D20C9D
:10751000F0CC303BD33C50ABE3D6A96805AD1BF6AD
:1075200066C93945C2A3A982EC20D513CEE898D606
:107530001FEB276BA7AC811C5BB67E1603227E1D5A
:107540006AB6D2B8BCE1374150566738B6B92EE5B5
:10755000D3090D74AE852FFCEA4641E06646538E92
:1075600067C373403A425C227A5F2C14E6BC0E2457
:10757000C982591DC18ED1E8A3300FA4C3A9D8A8D0
:107580007DB6490A60A8736E9DF389A37E9B1E5643
:107590007E8089A3320FC08B81CE156FD18041A32D
:1075A0005114DDC6E59C90163E7E5A86B16E99AEAA
:1075B00033922EAEBAE3862920DACAC73C0311897A
:1075C000A53490C32A1E6CB764BE88C0B14FF27256
:1075D0000214A764116F6BED8372B474A09F333BE8
:1075E0004667416D51ADD1AC0DE73126F6897A354C
:1075F000003970C88DA57B87A199426326D2DC191A
:107600005B03B40EC1183C26E23C2AFF218A9E028D
:10761000C4871EEE86A232473D36AD8B76126AB61F
:10762000663CAB29BB229F4EF16EDA4024416E7D51
:10763000A26D1F7C51AF2EF3D99180A91C1B7FBE78
:1076400040E9439FC20DF58567B41773B2791DEC0D
:10765000219EE3B813CD3EC24253B6F91C0347D274
:107660000AB071673CC4FA18078D8FCEF61080708F
:107670001BA71986368063B63C69A0538E6E25FE23
:10768000CF4D917EBC92821E4F70710665E10CD188
:10769000D4CE78D6E08B3D8D053ECD0C5FF1D42065
:1076A0002F5ED19537B58326F58B14BB5CC58794C7
:1076B000544F852F5CB8046906EE7F7C5D3E16E270
:1076C000862E25681C862D535A937706717899DD8E
:1076D00062E9F3DE6556F958C677C32D8147E0FFAE
:1076E0002D10E8F0B383F8C0DC62C6EC39091A73D8
:1076F000E00063A30DC521948400270DC641234BF0
:107700005EE03FED9C16DF74F9E2014EF8E8D172BD
:107710001B935B7B507CE66870B9ABE11EA6BED6BE
:10772000A5553C454586C4D0E684D0A768CA690300
:107730002BC8440EBCA1FA169BCECB38F6945BB393
:10774000EE7FA4C5B157A6CF8FC23E07D58FD3D841
:10775000F7982E9E6DE199848C1F48E6ABE760395F
:107760002E855050DD9106B2F3A766FA368BCF799D
:107770007E549CEDE5801B2C5D250F322D0BDB3BF1
:10778000E8EBE65BB51EAE2576197DB3B9A30F4FC6
:1077900098C1E03CA5320C49E5EB5B8AEA42C9A2FC
:1077A0003F8DE5E1C20AC49E181925C53D41FB1F66
:1077B000446269E5A08A03E9D3149E27FE4C3CB3DA
:1077C0003D2D621D62E0249A53C62ED9D877C3F3AB
:1077D0001DC45877F38A6753C250182352A752DF4B
:1077E00084C4B8A9783692E754DF06FAD74D07D19A
:1077F000DC16E65CFEDCE688671E699326AE6C400C
:10780000F1F340F33291CB6B910703CF3490AB157A
:107810005A5E5FADEAEA6E7F19A2BB7410D4C2EE65
:107820001183CD1595BB723CC4EC6B95ACB57277EA
:10783000F86E783070A32E9A65F8F4B9B995EABC61
:10784000A2118B81A6A87CB7902B19CF86E58874EE
:107850000344D2536502351FAA55FD2C0CA61EED1C
:10786000FDDB91FD02851EF92AE36523DE5E4E8F66
:1078700045872D296ED2B38D3A0F9B8174CF469DDB
:10788000DFC94525B7BC9C0F443F0E74A61E689601
:10789000AD09FD34D0F2FDAEC7CA9DA879B67459C2
:1078A0002176B42D36AA1AAEFF2832A2D5D0B874EC
:1078B0005162B603F18042FA249E393CBC65FA5706
:1078C00008319B8151FB5799B1FF3C06B386E122F9
:1078D00039FE27203692DF88E536A0EC486AB811D9
:1078E0001BADC227A5BE9EF381D305CD46F0ECD2D9
:1078F000273A8A9E79F4C5F7C8CB681E49D9D0F7D4
:10790000DFC9BE8E58AF6FF3897F88CD952EDD3FDE
:10791000971D25B6BA5835F462A3D4CABA45318C3E
:1079200032B5A4CEA94C365D3FBE88DE29DD104FAE
:107930005550D5F0A5472EC369203FEDC874A3FF6D
:107940005778FEF5A0A4CC54C6586A10519A2D8BD6
:1079500088F7B50DB38E56EA4C418B9F6844EF5CB7
:10796000F615EF5DFE5772169ED214FABFFF4EF663
:107970005B808CBD7EA21AF28E1CEF3966B3FE2CA2
:1079800036EA2A9E7D51CDEC9DA9033DD1A49A13E0
:10799000DA0D0D3C0BF700F9C921CBA3595E704AF3
:1079A0002F0C6193813E1A782B55C657B46890DC32
:1079B000894D6F1EEA0ACD1DAB73606A7D71E67D4D
:1079C00049376060E1F99432429B3D55CC592E8E87
:1079D0005372FE80E06BCF5CAB8744C0927926EE99
:1079E00006B1E98D0D9B0B75F65953B3F3117977F9
:1079F000EF05CF5DBEF3EBFD9A155EA870275E0321
:107A0000FE9D74E327C0B733AD995CF0A9E64B3B0C
:107A1000E2F40DD2AA293587F5C286738A9DD4393E
:107A2000B182341BA18939DD480E8BEEF6E6228F38
:107A30007A2F422C658FACDBDFF8F9D3EF817351DD
:107A4000C60A68C44C46EFE6C47F57ACBFD870D6B0
:107A5000CDF2C8C8A7E25C8E7722EF2ED7CE7C9EEF
:107A60007DE9C1E44E6E4A0B1B650263CBE5D98309
:107A70002129F406236891BF68469FBCBDB44E9C83
:107A800075C5AA2F7FE254A71B790CFA1653E44D53
:107A900017032B9E6FFD2EE6F7861F2F76D6E64B3B
:107AA0008A0BBA6CB1FE5232A4E3106FE66FDB8131
:107AB000E28D0AD28DCC5BC999E994CE9FF05C8EA1
:107AC000FC515DF415A29FC771D9ECAEFD93C810AF
:107AD0005577F1953C4A30702E27442FD96D792A7D
:107AE000113641E4A6A889235FF340F34CEDA2EAE6
:107AF0007C649E63B56D24C90659E6BC2187C9170D
:107B0000F1F864849E21B841D66A1F49E63357755F
:107B100050DBD32D2D3D8F34650CFDF89AE5F954DB
:107B200029765C81F27DA34F021F966778C0E8F149
:107B3000F6C8988E0A315FFE04379426D6C0CB6B08
:107B40001F41650A7E8AFDBAB1E7A79322F3BD877C
:107B500081F06BB228FD99BA8765CC03A30C6E5DEA
:107B60007D25CFC3C1A48169CA24B035F671798659
:107B7000178CD369449C96F2FB2FFA13FE01AAB32B
:107B8000F2CC51DE58B8D3FBA681FA8C7466E2AF12
:107B90005B1929DD86CFF7C4334DB9D45316818FD5
:107BA0004BF38A1748B427BFDD06FE015BCB6F3A63
:107BB00056BFE9E7B70D2BFC84E42D9DD9D5817E16
:107BC000F35D4FE9B753E627B487E659A15028146F
:107BD0000A85E2C7F0DFFF297E16C4F35FFFF94B89
:107BE000F1A3F8FFDA9142A15028140A8542A1506E
:107BF00028140A8542A15028140A8542A15028144D
:107C00000A8542A15028140A8542A15028140A85E9
:107C100042A15028140A8542A1502814BF167F03A0
:047C20000E2F4935A5
:107C240020030000E0010000200400002E000000FA
:107C34000A0000000D020000170000000A00000006
:107C44000201000004000000E001000085000000C3
:087C5400E00100000000000047
:0400000508000000EF
:00000001FF
